:1000000000800020BD010000595000002550000074
:10001000255000002550000025500000255000000C
:1000200025500000255000002550000059500000C8
:100030005950000025500000595000001550000094
:10004000595000005950000059500000595000000C
:1000500059500000595000005950000059500000FC
:1000600059500000595000005950000059500000EC
:1000700059500000595000005950000059500000DC
:1000800059500000595000005950000059500000CC
:1000900059500000595000005950000059500000BC
:1000A00059500000595000005950000059500000AC
:1000B000595000005950000059500000595000009C
:1000C000595000005950000059500000595000008C
:1000D000595000005950000059500000595000007C
:1000E000595000005950000059500000595000006C
:1000F00059500000D159000059500000955F000090
:10010000595000007164000059500000595000001F
:10011000595000005950000059500000595000003B
:100120005950000069090000990C00005950000066
:10013000595000005950000059500000595000001B
:10014000595000005950000059500000595000000B
:1001500059500000595000005950000059500000FB
:1001600059500000796700005950000059500000B4
:1001700059500000595000005950000059500000DB
:10018000595000005950000059500000114800001B
:1001900059500000595000005950000059500000BB
:1001A00059500000595000005950000059500000AB
:1001B000595000005950000059500000564B4CF265
:1001C000205210B51A804DF628121A8000BF00BFC9
:1001D00004F046FF514B4FF010621A60504A9A608B
:1001E000504ADA60A3F53043203B1A6812F480725B
:1001F00004D14D490A604FF4A8521A604B4B1A784B
:10020000110703D51A7842F008021A70484B2A22C7
:100210001A700023474A48499818884204D247492F
:10022000595899500433F5E7454A464B9A424FF0E6
:10023000000302D242F8043BF7E74349434A5958C6
:1002400099500433B3F5DE7FF7D1414B802103F899
:10025000011B40498B42F9D13F4B1A603F4B0A22A8
:100260001A70A3F5805324225A70A0221A709A792A
:100270009207FCD59A79D406FCD4394B9A7902F0CE
:100280000C02082AF9D103221A7140225A719A7974
:100290009006FCD5324B9A795106FBD5314A32494A
:1002A00011600221516020221A702D4B9B7903F0BE
:1002B0000C030C2BF9D12D4B2D4A1A602D4B2E4AD5
:1002C0001A6000225A60072243F8042C2B4AC3F814
:1002D0000C2D62B605F0D8F8134B1B68DA0705D56C
:1002E000274804F0F5FE274B274A1A60274B1B7856
:1002F0005B0609D5234C244A2368934204D1204845
:1003000004F0E6FE0023236007F00CFD04F0AEFECF
:1003100007F04CF8FEE700BF0E2005403080044097
:10032000823F04000100002B14D0034002D007409C
:1003300000E007406087FF1F7C88FF1FB8AD00000A
:100340007C88FF1F1091FF1F000000000082FF1F2C
:1003500000E400E05FE400E008ED00E0005006404B
:100360000040064044800440000003010480044033
:10037000C010050014E000E0FF760100000020201E
:1003800000DD68501CE00340A5C3945A00F007400C
:10039000FFFFFFFFFFFFFFFFFFFFFFFFFFFFFFFF6D
:1003A000FFFFFFFFFFFFFFFFFFFFFFFFFFFFFFFF5D
:1003B000FFFFFFFFFFFFFFFFFFFFFFFFFFFFFFFF4D
:1003C000FFFFFFFFFFFFFFFFFFFFFFFFFFFFFFFF3D
:1003D000FFFFFFFFFFFFFFFFFFFFFFFFFFFFFFFF2D
:1003E000FFFFFFFFFFFFFFFFFFFFFFFFFFFFFFFF1D
:1003F000FFFFFFFFFFFFFFFFFFFFFFFFFFFFFFFF0D
:10040000FFFFFFFFFFFFFFFFFFFFFFFFFEFFFFFFFD
:1004100010B5054C237833B9044B13B10448AFF33E
:1004200000800123237010BD7C88FF1F00000000A6
:10043000B8AD000008B5064B1BB106480649AFF33E
:1004400000800648036813B1054B03B1984708BD07
:1004500000000000B8AD00008088FF1F7C88FF1FEF
:10046000000000002DE9F04101210D2004F0D8FE2C
:100470006E4B6F4C6F4E20221A604FF4847006F062
:100480009DFF054602F088FA2846256002F017FA1B
:10049000FE2812D140F2DC5004F0E0FF4FF41D7052
:1004A00006F08CFF644904464FF4E13200F0AEFFE1
:1004B0003460306802F0B0F8FBE723685F4993F8D6
:1004C000A20004F015FE5E4B4FF496721A605D4B6D
:1004D000C0221A602368012193F8A20004F0A0FE54
:1004E0002368402193F8A20004F0B6FE0C2004F02B
:1004F0006FFB082004F096FB40F2DC5004F0AEFFE6
:10050000206802F09EF9430803F1376303F5D833FE
:10051000B3FBF0F005F006F8206802F0B4F920B162
:10052000236893F8A00005F0A9F8206802F0B5F957
:10053000430803F1376303F5D833B3FBF0F005F05C
:10054000DBFA206802F0B2F9430803F1B76303F560
:100550005843B3FBF0F005F0B1FD206802F09DF9BF
:1005600005461C2006F02AFF2A463749374D074624
:1005700003F03EFC20682F6002F063F980464FF4E0
:10058000107006F01BFF42463149074603F03AF867
:10059000304B58201F6006F011FF074600F096FB15
:1005A0002D4B2E491F60384600F0FCFC4FF41D70A7
:1005B00006F004FF20494FF4E132074600F026FF21
:1005C0002068376002F072F907464FF41D7006F09C
:1005D000F5FE3A462149064600F018FF204B2868F0
:1005E0001E60204E03F028FD286803F0EFFD3768F9
:1005F000286807F6F43703F0E9FC3368BB4203D2FE
:10060000286803F0E3FDF8E760210B4620680A46FE
:1006100002F0E3F800F082F923681B7E23B1012089
:10062000BDE8F04103F0F6BFBDE8F08184F00F4073
:10063000B488FF1F9888FF1FD890FF1F0000A041BB
:10064000A488FF1F9C88FF1FB890FF1FBC88FF1F56
:10065000A890FF1FB088FF1FAC88FF1FC890FF1F26
:10066000B888FF1FF488FF1F1C4B1A684FF6E8512B
:1006700001328A4270B51A601D462EDD184C23687F
:10068000D3F8AC0003F044FE23680C2690FBF6F68A
:10069000986803F033FEB0F5967F05DDB0F5167F60
:1006A000A8BF4FF4167001E04FF496700D4A23680E
:1006B0001268A0F596700A21414391FBF2F10A4AB3
:1006C00093F8A2001268514301F52071F6B291FB34
:1006D000F6F104F0C1FD00232B6070BDA888FF1F58
:1006E000B488FF1FA488FF1F9C88FF1F0F4B1A6848
:1006F000002A08DA0E49086801280DD00120086098
:1007000020200C4907E007D00949086820B10020E3
:10071000086009492020086001324FF6E8518A42FA
:10072000C8BF6FF031021A60704700BFA088FF1F7A
:100730006087FF1F84F00F4088F00F402DE9F843D9
:100740006B4E6C4D33686C4C93F8BC30DFF8C8814D
:100750006A4F8BB9286801F05FFF206801F05CFFE9
:10076000D8F8000003F0E8F9386803F02FFDFFF730
:100770007BFFFFF7BBFFE3E7D8F8000010B1036889
:100780009B689847386810B103689B689847286849
:1007900010B103689B689847206810B103689B6894
:1007A000984700F0D7F833681B7E0BB104F0A0F82F
:1007B0003368534A93F8BC30524C534F13F0040F34
:1007C00008BF1446514A97F8008013F0010F18BF74
:1007D000144613F0080F4E4B08F0010818BF1C46D2
:1007E0003068434D40218022002301F0F6FFB8F12C
:1007F000000F1ED13B78DB071BD5424B9C424FD1EB
:1008000004F008FF286802F063FB424B18684308B5
:1008100003F1376303F5D833B3FBF0F004F082FE45
:10082000286802F030F820B12B6893F8A00004F09B
:1008300025FF97F8008008F00108314D2B68284605
:100840009B689847A94680B1002213463068402132
:1008500001F0C3FF2368D3F800902B682846DB68BB
:100860009847C1B22046C847E7E7236820469B68FF
:10087000984780B1306840218022002301F0ADFF0D
:10088000D9F800301D6823682046DB689847C1B25C
:100890001B48A847E9E7FFF7E7FEFFF727FF9FE7B9
:1008A0001A4B9C4210D105F09FF9286802F010FB0A
:1008B000184B1868430803F1376303F5D833B3FBCB
:1008C000F0F005F019F9B4E7114B9C42B1D105F0F5
:1008D00061FC286802F0FCFA0E4B1868430803F12B
:1008E000B76303F55843B3FBF0F005F0E7FBA0E76F
:1008F000B488FF1F9888FF1FB888FF1FBC88FF1FA0
:10090000D890FF1FA890FF1FA490FF1FB890FF1F53
:10091000C890FF1F0091FF1FB088FF1F08B5094B4B
:100920004FF000721A604FF080621A60064B1B682D
:1009300093F82500054B187004F00EFA044B0122C1
:100940001A7008BD04E100E0B488FF1FC088FF1FD3
:10095000C288FF1F034B4FF000721A604FF0806295
:100960001A60704784E100E070B5B24C23780F2B19
:1009700000F28781DFE813F0210036004B006000B1
:1009800075008A009F00B400C900DE001D0134011B
:10099000010168014A011000A74D287804F024FAEB
:1009A000A64B1B68D3F8AC20132101FB02001426D0
:1009B00090FBF6F2C3F8AC20D8E09F4D287804F005
:1009C00013FA9E4B1B681A6B452101FB0200462659
:1009D00090FBF6F21A6393F82500287004F0BCF936
:1009E00001234CE1944D287804F0FEF9934B1B68E9
:1009F0005A6B452101FB0200462690FBF6F25A6332
:100A000093F82600287004F0A7F9022337E18A4DF5
:100A1000287804F0E9F9894B1B689A6B452101FBA2
:100A20000200462690FBF6F29A6393F8270028709E
:100A300004F092F9032322E17F4D287804F0D4F9E1
:100A40007E4B1B68DA6B452101FB0200462690FBBA
:100A5000F6F2DA6393F82800287004F07DF9042395
:100A60000DE1754D287804F0BFF9744B1B681A6CC2
:100A7000452101FB0200462690FBF6F21A6493F82A
:100A80002900287004F068F90523F8E06A4D2878F9
:100A900004F0AAF9694B1B685A6C452101FB02005E
:100AA000462690FBF6F25A6493F82A00287004F068
:100AB00053F90623E3E0604D287804F095F95F4B85
:100AC0001B689A6C452101FB0200462690FBF6F25A
:100AD0009A6493F82B00287004F03EF90723CEE0C7
:100AE000554D287804F080F9544B1B68DA6C452189
:100AF00001FB0200462690FBF6F2DA6493F82C0024
:100B0000287004F029F90823B9E04B4D287804F047
:100B10006BF94A4B1B681A6D452101FB0200462602
:100B200090FBF6F21A6593F82D00287004F014F982
:100B30000923A4E0404D287804F056F93F4B1B6888
:100B40005A6D452101FB0200462690FBF6F25A65DC
:100B50003B4A1178092907D9987B28700021117028
:100B600004F0FAF80C238AE00131117093F82400A4
:100B7000287004F0F1F8002381E02F4D287804F06C
:100B800033F92E4B1B681A69632101FB02006426AE
:100B900090FBF6F2597B1A612A4A52F83120012162
:100BA00082F8801093F89500287004F0D5F80A2395
:100BB00065E0214D287804F017F9204B1B68D3F825
:100BC0009C2002EBC20210440A2190FBF1F2C3F810
:100BD0009C2093F89400287004F0BEF80B234EE09C
:100BE000154D287804F000F9144B1B68D3F89820B1
:100BF00002EBC20210440A2190FBF1F2C3F89820E4
:100C00001879287004F0A8F80E2338E00A4D2878E7
:100C100004F0EAF8094B1B689A68312101FB0200D5
:100C2000322690FBF6F29A60987B287004F094F8D4
:100C30000D2324E0C288FF1FC088FF1FB488FF1F58
:100C4000C188FF1F38A90000104D287804F0CCF8A7
:100C50000F4B1B685A69632101FB0200642690FB5D
:100C6000F6F2597B5A610B4A52F83120012182F881
:100C7000001193F8A800287004F06EF80F23237079
:100C800070BD0220BDE8704003F04EBBC088FF1F5E
:100C9000B488FF1F38A90000FFF766BE38B50446C8
:100CA00008460D4607F085F9236802465B68204632
:100CB0002946984738BD38B50446FFF7EFFF05468B
:100CC000204606F09FFB284438BDFFFF38B50025BD
:100CD00004460571457180F85450044914220630C9
:100CE00007F086F92565204638BD00BFF88B000067
:100CF0000079704790F85520044B53F832200123B7
:100D000082F8803003711846704700BF38A9000090
:100D100038B5084B90F8552053F832300124054679
:100D200083F800410A2004F099FB00232B71204630
:100D300038BD00BF38A900004079704706307047C1
:100D4000006D704738B50446006803681B6A984711
:100D50002046FFF7DDFF94F856200E4B53F8323053
:100D6000012583F880500A2004F078FB2046FFF725
:100D7000C1FF2068084B20221A6003684FF4164117
:100D80009B69984740F2EE2004F068FB84F85450C9
:100D900038BD00BF38A9000084F00F4070B504468C
:100DA000006803681B6A98472046FFF7B1FF94F874
:100DB00056200E4B53F83230012283F800210A20CE
:100DC00004F04CFB2046FFF795FF2568084B2022D6
:100DD0001A602B689E69074B186801F067FD014691
:100DE0002846B047002384F8543070BD38A900006D
:100DF00088F00F40B488FF1F10B58EB0322201A8D2
:100E00000C4607F0F5F800233A2101A88DF835309B
:100E100007F0B0F8014608B9207003E02046013120
:100E200007F0BFF80EB010BD2DE9F84300250746C6
:100E3000884691460D702C462E46386803689B689C
:100E4000984748B338680368DB689847C0B20EB962
:100E500045282DD001360D28F6B203D1002308F81D
:100E6000043009E009F1FF339C42F7D008F8040090
:100E70000134E4B20025E0E7386803689B689847CE
:100E800038B138680368DB6898470A2004F0E6FA4E
:100E9000F2E70120BDE8F88301350A20EDB204F045
:100EA000DDFA312DC9D9201C18BF0120BDE8F88317
:100EB0003046BDE8F883FFFF70B504462546067945
:100EC000FFF740FF002355F81A0B0E496371FFF737
:100ED000F2FE204629463222FFF7A6FF38B1284607
:100EE0000949022207F06DF808B9012300E0002348
:100EF00063712046FFF752FF16B92046FFF708FF3F
:100F0000607970BD1E8C00001B8C0000437970B5A9
:100F10000446F3B190F854600EB9FFF713FF25466D
:100F20000C4955F81A0BFFF7C6FE32222946204617
:100F3000FFF77AFF20462946FFF75EFFA01D2946EE
:100F4000142207F055F826B92046BDE87040FFF797
:100F500025BF70BD218C0000437970B50446EBB10C
:100F600090F854600EB9FFF7EDFE25460C4955F890
:100F70001A0BFFF7A0FE322229462046FFF754FF46
:100F800020462946FFF738FF284606F0B9FE2065BF
:100F900026B92046BDE87040FFF700BF70BD00BF16
:100FA0002A8C000070B52B4D01600446286801F0C2
:100FB00086FC032804D1212384F85530172306E04A
:100FC0000438012837D8032384F85530182384F8CF
:100FD000563094F85600012104F022F994F8562076
:100FE0001D4B53F83230012183F8001194F855005D
:100FF00004F016F92046FFF77DFE2046FFF75CFF60
:10100000637933B32046FFF79DFE2046FFF7A4FF28
:101010002046FFF77BFF2046FFF7C0FE2046FFF784
:1010200069FE2468286823689E6901F03FFC014638
:101030002046B0470DE00A2003F076F9074B06344E
:1010400003F1140253F8041B44F8041B9342F9D132
:1010500070BD70BDB488FF1F38A90000338C00003C
:10106000F8B5437904460F4643B390F854600EB97F
:10107000FFF768FE25463A461149206806F0D8F980
:1010800055F81A0B0F49FFF709FE20462946322270
:10109000FFF7CAFE60B128460B49022206F091FF15
:1010A00030B9A01D3946142206F0A2FF012500E048
:1010B000002516B92046FFF771FE2B461846F8BDED
:1010C000478C0000188C00001B8C0000437970B521
:1010D00004460D462BB390F854600EB9FFF732FE6C
:1010E0002A4625461049206806F0A2F955F81A0B41
:1010F0000E49FFF7D3FD204629463222FFF794FE22
:1011000048B128460A49022206F05BFFD0F10105EA
:1011100038BF002500E0054616B92046FFF73EFE21
:101120002B46184670BD00BF098C0000188C0000CB
:101130001B8C0000F8B5437904460F4623B390F8A2
:1011400054600EB9FFF7FEFD25463A460F49206868
:1011500006F06EF955F81A0B0D49FFF79FFD204672
:1011600029463222FFF760FE40B128460949022293
:1011700006F027FF10B92765012500E0002516B904
:101180002046FFF70BFE2B461846F8BD528C000098
:10119000188C00001B8C0000F8B5437904460F46FC
:1011A00000F11A050BB9837615E090F854600EB97A
:1011B000FFF7C8FD39462068FFF770FD0749206832
:1011C000FFF76CFD204629463222FFF72DFE16B9A7
:1011D0002046FFF7E3FD2846F8BD00BF188C00004D
:1011E0001FB500230446C360036101214FF4BF70A3
:1011F00006F08EFD206050B90A49684606F0C4F931
:10120000684603F0D5F8684606F07EF907E04FF42B
:10121000BF70042106F07CFD42236060A36020467D
:1012200004B010BD5F8C00000A23034AB1FBF3F148
:10123000B2FBF1F38360704730D4050010B504466B
:10124000006806F09DFD606806F09AFD204610BD1E
:1012500003690268D154084A03691168426842F878
:1012600023105A1CB2F5BF7FA5BF6FF4BE729B1846
:1012700002610361704700BFF488FF1FC268036901
:101280009A42CABFC2F5BF72C2EB0300D0187047C2
:1012900038B50D460446FFF7F1FF854204DB062012
:1012A00003F042F8002038BDE16823682944B1F515
:1012B000BF7FA8BFA1F5BF71585C38BDC368006986
:1012C0005A1E48BF03F27D12131A58425841704704
:1012D0000023C3600361704738B50D460446FFF72D
:1012E000CDFF854204DD0820BDE8384003F01CB87E
:1012F000E1682944B1F5BF7FA8BFA1F5BF71E160E6
:1013000038BDFFFF38B50B4B1D6883680446ED1AE6
:101310002046FFF7B3FF00280ADDE268636853F850
:101320002230AB4204D820460121FFF7D5FFEFE77A
:1013300038BD00BFF488FF1F014B0360704700BF3A
:10134000B08C0000014B0360704700BFB08C000000
:1013500010B5034B0360044606F032F8204610BD7A
:10136000B08C000010B5034B0360044606F028F86B
:10137000204610BDB08C000030B585B004AC04E947
:101380000E00089C34B940681A4905B0BDE83040E9
:1013900006F04EB89DF80430022B08D0032B1ED166
:1013A000154994F80421406806F042F81BE094F8CF
:1013B000022194F80431012A03D140680F49E278F0
:1013C0000AE0022A06D1E278257940680B4902EB4F
:1013D000052201E040680A4906F02AF803E00948BE
:1013E000094906F025F8204605B0BDE8304006F072
:1013F000C7BC00BFE08C0000088D0000EB8C000033
:10140000F68C0000D890FF1F0E8D000010B5074C21
:101410000460002480F86D4180F8734241604266A8
:1014200080F8484080F8604010BD00BFD08C0000BC
:101430002DE9F041204B214F1B88D7F800808AB05E
:101440000024ADF8143002236D460093404605ABEE
:101450000321FE228DF81D40089402F02CFD45F872
:10146000044B07AE034696E8070085E807004046B0
:1014700019462246234602F0D9FC3F688DF81940F0
:1014800003211E238DF81830009106AB3846FE224A
:101490008DF81A4002F00FFD0094034696E807000D
:1014A00085E80700194638462246234602F0BEFC6E
:1014B0000AB0BDE8F08100BFC08C0000BC88FF1FEF
:1014C0002DE9F0432F4FDFF8C0803B88D8F800901B
:1014D0008BB00025ADF8143002236C4600934846CB
:1014E00005AB0321FE228DF81D50089502F0E3FCA8
:1014F00044F8045B07AE034696E8070084E807005B
:10150000484619462A462B4602F090FC3B46D8F83E
:10151000009033F8022FADF8182003279B788DF840
:101520001A30394606AB00974846FE2202F0C3FC4B
:101530000095034696E8070084E8070048461946E8
:101540002A462B4602F072FCD8F800800097FF2351
:101550008DF819300F238DF81A30394606AB404606
:10156000FE2202F0A8FC0095034696E8070084E8F6
:101570000700194640462A462B4602F057FC0BB09E
:10158000BDE8F083C08C0000BC88FF1F0A4B10B57B
:10159000044618680023C218013300210A2B82F880
:1015A0008A10F8D1054B186802F010FD60680449F4
:1015B000FFF781FB10BD00BFB488FF1FBC88FF1F71
:1015C0003A8D00002DE9F341674D684904464068B3
:1015D00005F02EFF2868666801F071F9644902463B
:1015E000304605F025FF2868666801F06EF961490C
:1015F0000246304605F01CFF2868666801F06BF96A
:101600005D490246304605F013FF2868D4F804808F
:1016100001F06AF90746286801F06CF90646286867
:1016200001F06EF93346554900903A46404605F0C0
:10163000FFFE2868666801F06FF95149024630469E
:1016400005F0F6FE286801F061F910B160684D49B7
:1016500001E060684C4905F0EBFE4C496068FFF71B
:101660001DFB2868666801F05DF94949024630466D
:1016700005F0DEFE2868676801F0E6F8064628688F
:1016800001F0DFF8324603464249384605F0D0FE05
:101690002868676801F0DEF80646286801F0EDF872
:1016A000324603463C49384605F0C2FE2868666863
:1016B00001F0E6F839490246304605F0B9FE2868DF
:1016C000666801F0E0F8364B364A3749002818BF03
:1016D0001A46304605F0ACFE34496068224EFFF7EA
:1016E000DDFA2868D4F8048001F0DAF807462868A3
:1016F0002F4D01F0D2F82F4903463A46404605F0F7
:1017000097FE2868FFF718FB38B32B496068FFF78E
:10171000D2FA3068D4F8048001F0CBF8074630687C
:1017200001F0C4F83A4603462449404605F080FEDD
:1017300028686668FFF702FB21490246304605F03B
:1017400077FE28686468FFF7FBFA1E4902462046C8
:1017500002B0BDE8F04105F06BBE60681A49FFF7C2
:10176000AAFA02B0BDE8F081B488FF1F7E8D0000A8
:101770009B8D0000AB8D0000C68D0000DB8D00004E
:10178000F78D00001A8E0000518E0000888E000038
:10179000B08E0000568F0000C98E0000EF8E000052
:1017A000778D00007B8D0000088F0000218F0000E6
:1017B000AC88FF1F488F0000768F0000A58F0000C7
:1017C000CE8F0000EA8F0000089000002DE9F04164
:1017D0006A4D2B680446D3F8AC0002F099FD6849C5
:1017E0000746606805F024FE2B68D4F804809868EA
:1017F00002F084FD0A2690FBF6F26249404605F0AD
:1018000017FE97FBF6F206FB12735F4960685F4FA5
:1018100005F00EFE2B685E49D3F8A420606892FBA9
:10182000F6F205F005FE2B685A49D3F89C20606853
:10183000594E05F0FDFD2B685849D3F89820606893
:1018400005F0F6FD2B6856491A7B6068002A0CBF2C
:101850003A46324605F0ECFD2B6852491A69606839
:1018600005F0E6FD2B6850495A691B696068D21A79
:1018700005F0DEFD2B684D491A7E6068002A0CBF1A
:101880003A46324605F0D4FD2B684949DA6960686A
:1018900005F0CEFD2B6847491A6A606805F0C8FD5F
:1018A0004549606805F0C4FD444B45491A786068B5
:1018B00005F0BEFD434B44491A78606805F0B8FD59
:1018C000424B43491A78606805F0B2FD60684149AF
:1018D00005F0AEFD00262B68334493F88A201AB138
:1018E00060683D4905F0A4FD01360A2EF3D1606819
:1018F0003A4905F09DFD012628686768821992F82B
:101900007F1006F10B0250F8228049B101F004F873
:101910000146404602F001FD31490346384608E0E1
:1019200000F0FAFF0146404602F0F7FC2D4903465D
:1019300038463246013605F07BFD0B2EDCD12A4DB0
:101940002868FFF7F9F990B128496068FFF7B3F903
:1019500028686468FFF7CCF9254B264A26490028F9
:1019600018BF1A462046BDE8F04105F061BD606829
:101970002249FFF7A0F9BDE8F08100BFB488FF1F3E
:101980003D9000004C9000006B9000007B8D0000AB
:101990008C900000B6900000778D0000D69000007B
:1019A000F4900000179100003E9100006891000043
:1019B0008A910000AB910000CC910000F490FF1FD1
:1019C000E8910000C388FF1F0E920000F590FF1FF2
:1019D0003492000059920000C18E00007A920000FB
:1019E00089920000B9920000AC88FF1FD8920000D5
:1019F0003690000039900000079300000890000026
:101A000038B5184B45680446186800F064FF16495D
:101A10000246284605F00CFD6068144905F008FDF3
:101A20006068134905F004FD6068124905F000FD87
:101A30006068114905F0FCFC6068104905F0F8FC8D
:101A400060680F4905F0F4FC60680E4905F0F0FC91
:101A500060680D4905F0ECFC60680C49BDE8384051
:101A600005F0E6BCB488FF1F239300004D930000EF
:101A70001E940000319400003E9400005794000032
:101A800079940000A5940000C3940000E294000043
:101A900070B5294D46680446286800F01CFF2749A8
:101AA0000246304605F0C4FC6068254905F0C0FCDC
:101AB0006068244905F0BCFC6068234905F0B8FC67
:101AC0006068224905F0B4FC6068214905F0B0FC6B
:101AD0006068204905F0ACFC1F49606805F0A8FC6F
:101AE0002868666800F015FF1C490246304605F07C
:101AF0009FFC2868666800F00CFF194902463046D2
:101B000005F096FC6068174905F092FC606816497C
:101B100005F08EFC6068154905F08AFC6068144980
:101B200005F086FC6068134905F082FC6068124984
:101B3000BDE8704005F07CBCB488FF1F2393000013
:101B4000309500006F95000083950000AA95000075
:101B5000CF95000008960000199600002C96000012
:101B600059960000A1960000E49600006B970000D3
:101B7000A9970000E6970000189800004068014906
:101B800005F056BC4B9800002DE9F04F03298BB0AF
:101B900004460F4602D0FFF7F1FF5BE0006D06F050
:101BA000AFF88046606D06F0ABF82C4B5FFA88F812
:101BB00081464146186800F0BDFE10B960682849AA
:101BC00004E0B9F5805F04DB6068264905F030FC6D
:101BD00040E0DFF898A0244BDAF800B01B88ADF89D
:101BE0001430022300256C4600933946424605AB6B
:101BF00058468DF81D50089502F05DF944F8045BD5
:101C000007AE034696E8070084E8070019465846E1
:101C10002A462B4602F00AF98DF819904FEA292935
:101C20008DF81A90DAF8009000971E238DF818307E
:101C30003946424606AB484602F03DF90095034658
:101C400096E8070084E80700194648462A462B46CE
:101C500002F0ECF80BB0BDE8F08F00BFB488FF1FB6
:101C60009C980000E8980000C08C0000BC88FF1F12
:101C70002DE9F04302298BB00C4602D0FFF77EFF1E
:101C800041E0224F006D06F03BF8214BD7F8009061
:101C90001B88ADF8143000258046009403216C4663
:101CA000FE2205AB48468DF81D50089502F003F959
:101CB00044F8045B07AE034696E8070084E8070093
:101CC000194648462A462B4602F0B0F83F688DF880
:101CD000198003211E238DF818300091FE2206ABD7
:101CE0004FEA282838468DF81A8002F0E4F800956B
:101CF000034696E8070084E80700194638462A4656
:101D00002B4602F093F80BB0BDE8F083BC88FF1FB0
:101D1000C08C00002DE9F041042988B0044602D0AF
:101D2000FFF72CFF5FE0006D05F0EAFF0546606DF0
:101D300005F0E6FF8046A06D05F0E2FFFF280746AC
:101D40004CDC2A4EEDB2306829465FFA88F800F084
:101D5000F1FD18B300238DF815300693244B8DF850
:101D600010801E688DF811700223032100932A460B
:101D700004AB30468DF8141002F09DF86B46054612
:101D800043F8044B08AC14E9070083E80700304629
:101D9000294601221E2302F049F824E0306800F0B1
:101DA000C1FD85421AD10A2384F86830032384F8E0
:101DB0006A300223306884F8695004F1680104F540
:101DC000B77284F86A3184F86B8084F86C7001F023
:101DD000BDFA6068074994F8722202E0606805491C
:101DE000082205F025FB08B0BDE8F081B488FF1F8C
:101DF000BC88FF1F088D0000F0B5032989B0044698
:101E000002D0FFF7BBFE5AE0006D2E4E05F078FFC2
:101E1000C5B2606D05F074FF2946C7B2306800F0A6
:101E200089FD18B300238DF815300693264B8DF8E5
:101E300010701F680221012600912A4604AB384623
:101E40008DF814108DF8116002F035F86B460546D8
:101E500043F8044B08AC14E9070083E80700384650
:101E6000294632461E2301F0E1FF28E0306800F0E9
:101E700059FD85421ED10A2384F86830022384F874
:101E80006A3084F86A31012384F86C30306884F851
:101E9000695004F1680104F5B77284F86B7001F0C1
:101EA0002DF86068094994F8712194F8723205F0B0
:101EB000BFFA04E060680649082205F0B9FA09B0E3
:101EC000F0BD00BFB488FF1FBC88FF1FEB8C000073
:101ED000088D00002DE9F041042988B0044602D0A5
:101EE000FFF74CFE5FE0006D304F05F009FFC5B213
:101EF000606D05F005FF5FFA80F8A06D05F000FF4A
:101F000029460646386800F015FD28B300238DF8F1
:101F100015300693264B8DF8116036128DF812603D
:101F20001E688DF81080032100912A4604AB3046CC
:101F30008DF8141001F0BFFF6B46054643F8044BC3
:101F400008AC14E9070083E807003046294601225F
:101F50001E2301F06BFF26E0386800F0E3FC8542A9
:101F60001CD10A2384F8683084F86C60032336128D
:101F7000386884F86A3004F1680104F5B77284F8AF
:101F8000695084F86A3184F86B8084F86D6001F0E0
:101F9000DDF96068074994F8722202E0606805493B
:101FA000082205F045FA08B0BDE8F081B488FF1FAB
:101FB000BC88FF1F088D00002DE9F041032988B07F
:101FC0000446884602D0FFF7D9FD5CE0006D2F4E35
:101FD00005F096FEC5B2606D05F092FE2946C7B2C7
:101FE000306800F0A7FC10B300238DF8153006937D
:101FF000274B8DF810701E68022100912A4604AB11
:1020000030468DF811108DF8141001F054FF6B4616
:10201000054643F8044B08AC14E9070083E80700C1
:102020003046294601221E2301F000FF2BE03068D4
:1020300000F078FC854221D10A2384F8683002231D
:1020400084F86A3084F86C30306884F8695004F1A0
:10205000680104F5B77284F86A8184F86B7000F047
:102060004DFF94F8713194F872216068094903EBCF
:10207000022294F8723205F0DBF904E06068064948
:10208000082205F0D5F908B0BDE8F081B488FF1F3B
:10209000BC88FF1FEB8C0000088D0000022938B5BA
:1020A000044604D02046BDE83840FFF767BD056D03
:1020B0000E49284605F06BFF40B90D4B186800F03B
:1020C00007FF60680B49FEF7F6FD38BD28460A4950
:1020D00005F05DFF0028E5D1054C206800F0D8FE32
:1020E0002068BDE8384000F001BF00BF50990000F3
:1020F000B488FF1F5499000059990000032970B556
:1021000004461AD1056D6B49284605F040FFC8B951
:10211000656D6949284605F03AFF18B9674B0121FA
:10212000186807E06649284605F031FF014620B9E6
:10213000624B186800F0AAFB71E02046BDE87040D1
:10214000FFF71CBD28465F4905F021FFA8B9656D62
:102150005949284605F01BFF18B9584B012118684A
:1021600008E05749284605F012FF01460028E4D14F
:10217000524B186800F0EDFB51E02846524905F03B
:1021800006FF48B94D4B606D1D6805F0B9FDC1B241
:10219000284600F088FB42E028464C4905F0F7FE4F
:1021A000002841D1606D05F0AFFDCF28054602DD66
:1021B0006068474935E0474B013093FBF0F005F08C
:1021C0003FFB454905F044FC0021064605F03EFD75
:1021D00028B130464FF07C5105F07EFA04E03046DD
:1021E0004FF07C5105F076FA05F044FD3B4A03467A
:1021F0004FF4165110685943FEF768FF10B160683C
:10220000374901E06068374905F012F92B4BE9B214
:10221000186800F051FB60683349FEF74CFD6068B8
:102220003249FEF748FD70BD2846314905F0AFFE42
:1022300070B92A4B616D1868FEF712FF10B1606823
:102240002C4901E060682C49BDE8704005F0F0B809
:1022500028462A4905F09BFEC0B9606D05F050FD87
:1022600042F20F739842014602DD60682449EBE7B1
:102270001A4D2868FEF75EFF0028E3D028686468DE
:10228000FEF75EFD1F49024620460FE028461E4924
:1022900005F07DFE00287FF450AF104B616D18688B
:1022A0006568FEF779FF194902462846BDE8704087
:1022B00005F0BEB85D99000069990000B488FF1F61
:1022C0006D990000709900008099000088990000C5
:1022D0008F99000080841E0000001646AC88FF1F06
:1022E000DB990000FA990000199A00005499000047
:1022F0003D9A0000449A00004C9A0000529A000057
:10230000599A0000A79A0000DE9A0000E89A00009F
:10231000022970B504460D4608D1006D3C4905F010
:1023200036FE002849D102F02BF96BE0032944D195
:10233000056D3849284605F02AFE48B9364B606DD0
:102340001D6805F0DDFC0146284600F0BBFA59E0A7
:102350002846324905F01BFE48B92F4B606D1D68B9
:1023600005F0CEFC0146284600F0B2FA4AE02846C5
:102370002B4905F00CFE48B9274B606D1D6805F030
:10238000BFFC0146284600F0CAFA3BE02846254932
:1023900005F0FDFDB0B9656D2349284605F0F7FD50
:1023A00008B9282005E02846204905F0F0FD48B985
:1023B0001E20012102F0CAF824E0206D1C4905F01E
:1023C000E6FD20B12046BDE87040FFF7D7BB052DE4
:1023D000F8D1114D606D2E6805F092FCC1B2304607
:1023E00000F085FAA06D2E6805F08AFCC1B2304677
:1023F00000F083FAE06D2D6805F082FCC1B228463A
:1024000000F081FA60680B49FEF755FC70BD00BF13
:10241000F39A0000FA9A0000B488FF1F059B0000A1
:10242000139B0000239B00002E9B0000339B0000A9
:10243000399B000054990000F8B501230B7090F807
:1024400048303F2B84BF03F1FF3380F8483090F8C9
:10245000482002440023137204460E46012294F8D9
:102460004800D9B288420CD92144097A202905D1E3
:102470002AB9327801323270012200E000220133A1
:10248000EDE73378052BA8BF0523337004F1080569
:10249000002384F8603094F860703378BB421CD914
:1024A0002846202194F8482005F072FC30B904EB4E
:1024B00087030137DD6484F86070ECE7A84201D13E
:1024C0000135E8E704EB87070023FD64054605F8BE
:1024D000013B94F860300133DBE7E46C3E49204671
:1024E00005F055FD002859D020463C4905F04FFD28
:1024F000002855D020463A4905F049FD002851D022
:102500002046384905F043FD00284DD02046364985
:1025100005F03DFD002849D02046344905F037FD3F
:10252000002845D02046324905F031FD002841D031
:102530002046304905F02BFD00283DD020462E498D
:1025400005F025FD002839D020462C4905F01FFD57
:10255000002835D020462A4905F019FD002831D041
:102560002046284905F013FD00282DD02046264995
:1025700005F00DFD50B32046244905F008FD38B3A1
:102580002046234905F003FD20B32046214905F0EC
:10259000FEFC002814BF01201120F8BD0220F8BD68
:1025A0000320F8BD0420F8BD0520F8BD0620F8BDC5
:1025B0000720F8BD0820F8BD0920F8BD0A20F8BDA5
:1025C0000B20F8BD0C20F8BD0D20F8BD0E20F8BD85
:1025D0000F20F8BD1020F8BD3C9B0000419B00007F
:1025E000459B00004C9B0000529B0000649B000038
:1025F0005A9B0000609B0000699B0000709B0000DC
:10260000789B00000C9B00007D9B0000819B0000DC
:10261000859B0000899B000013B504466068036831
:102620009B689847002800F0848060680368DB6836
:102630009847C0B20D28F1D00A2894F8483001D14B
:10264000012B01D83F2B6ED120460DF10701FFF77A
:10265000F3FE112860D8DFE800F06C090D111519A0
:102660001D2125292F353B41474D53592046FFF762
:1026700085FA54E02046FFF70BFA50E02046FFF7BA
:10268000BFF94CE02046FFF7A1F848E02046FEF7EE
:1026900099FF44E02046FEF779FF40E02046FEF730
:1026A0000FFF3CE02046FEF7C3FE38E020469DF8D1
:1026B0000710FFF7DDFA32E020469DF80710FFF71C
:1026C00063FA2CE020469DF80710FFF7E7FC26E0B0
:1026D00020469DF80710FFF71BFE20E020469DF8DE
:1026E0000710FFF70BFD1AE020469DF80710FFF7D3
:1026F00011FB14E020469DF80710FFF7EBFB0EE0FE
:1027000020469DF80710FFF777FB08E020469DF86C
:102710000710FFF751FC02E00D2001F005FE002339
:1027200084F8483005E05A1C234484F84820187285
:1027300074E702B010BD0022026042608260704700
:102740000068704730B5044685B008200D4605F096
:102750000FFB50B90C49684604F016FF684601F0BB
:1027600027FE684604F0D0FE0CE000224260A2681A
:10277000056012B9A060606001E05060A06023684D
:102780000133236005B030BD8D9B0000406800B16F
:102790000068704738B504460D46002D63680DDDAE
:1027A00063B1186805F0ECFA60684368636005F08F
:1027B000E7FA2368013B2360013DEEE703B9A3601C
:1027C00038BD0168FFF7E6BF10B50446FFF7F9FF13
:1027D000204610BD0121FFF7DDBF70B504461E463F
:1027E00094F8C03080F8C110154690F8BD000BB1C8
:1027F000C943C9B202F030FD94F8C03084F8C35028
:1028000094F8BE0013B1ED43E9B200E0294602F0AE
:1028100023FD94F8C03084F8C26094F8BF0013B16F
:10282000F643F1B200E03146BDE8704002F014BD5D
:1028300090F8C100704790F8C300704790F8C2004C
:102840007047D0F8C800704790F8C40070470B205C
:1028500001F048BE90F8CC00704738B505460846F0
:1028600085F8CC100C4601F047FD2146C5F8D00094
:102870000C20BDE8384001F035BED0F8D0007047DC
:1028800090F8D400704790F8D60070470A46172099
:10289000012102B10A4601F0D5BDD0F8D800704739
:1028A00090F8D70070470F2001F01CBED0F8E00070
:1028B000704790F8DC007047102001F013BED0F88C
:1028C000E4007047002001F027BED0F8E800704710
:1028D000022001F021BE90F8F100704780F8F1105D
:1028E0000A20172101F0FEBD90F8F2007047042085
:1028F00001F0F8BD90F8F3007047052001F0F2BD3B
:1029000090F8F4007047062001F0ECBD90F8F0005C
:102910007047D0F8EC007047D0F8F80070471A20E4
:1029200001F0FABD90F8D500704780F8D5100E2060
:1029300001F0D8BD59B10023C21892F88A208A420A
:1029400003D001330A2BF7D101E0012070470020AA
:1029500070470A461720002101F074BD90F8F51069
:1029600010B50446B1B9D0F8E43090F8A100032BBB
:1029700002D102F055FC07E0012102F051FC94F86D
:10298000A100012102F02CFC322002F067FD01239E
:1029900084F8F53010BDFFFF2DE9FF4104460A2001
:1029A00001F044FD172884F8F10003D020461721D8
:1029B000FFF794FF002001F03FFDC4F8E40002207F
:1029C00001F03AFDC4F8E8000D2001F02FFD84F875
:1029D000D4000C2001F02AFD84F8CC0001F08CFC1E
:1029E000C4F8D0000B2001F021FD84F8C40001F0F0
:1029F00069FC0121C4F8C800172001F005FD003072
:102A000018BF012084F8D6000E2001F00FFD84F8D5
:102A1000D5000F2001F00AFD84F8D70001F052FC28
:102A2000C4F8D800102001F001FD84F8DC0001F0AA
:102A300049FCC4F8E000042001F0F8FC84F8F2003E
:102A4000052001F0F3FC84F8F300062001F0EEFC11
:102A5000002184F8F40084F8BC10172001F0D4FCA5
:102A6000003018BF012084F8F00010B140F6FF7369
:102A700001E040F2FF33C4F8EC30D4F8E83003F062
:102A800001022273C3F3400222765A0701D5322392
:102A900004E01B074CBF4A234FF0FF330025C4F866
:102AA000A43084F8F5501A2001F0C6FCD4F8E830C0
:102AB000C4F8F80013F0160F0CBF0023012384F8AC
:102AC000C0304FF44873C4F8B0304FF49663C4F884
:102AD000B43040F2DC53C4F8B8300A20012105F0CC
:102AE00017F9206050B9DA49684604F04DFD684690
:102AF00001F05EFC684604F007FDC5E1D4F8E4701F
:102B0000032F79D102234FF0040884F8A030404607
:102B1000012184F8BD8002F083FB052084F8BE000B
:102B2000012102F07DFB062084F8BF00012102F0A4
:102B300077FB2A46772320463321FFF74EFE1220EB
:102B40000121607302F06CFB2520A07302F094F861
:102B500019236061637620610F230B20A376012186
:102B600084F8A200242602F05BFB1D2084F8A860F4
:102B7000207102F081F8A06094F8A80002F07CF8BF
:102B80001A2384F824301C2384F82530152384F874
:102B90002630102384F827301F2384F8A130C4F88E
:102BA000AC002946092084F8286084F8296084F85C
:102BB0002A6084F82B6084F82C6084F82D6084F8F7
:102BC000946084F8956002F02BFB2020294602F0E7
:102BD00027FB3846294602F023FB0C20012102F096
:102BE0001FFB9C4B80221A601320012102F018FB6E
:102BF000994BC3F800800AE1042F70D1022384F8B6
:102C0000A030384684F8BD70012102F009FB052090
:102C100084F8BE00012102F003FB062084F8BF0007
:102C2000012102F0FDFAFF222B4620462946FFF73C
:102C3000D4FD1E206073012102F0F2FA1D20A07362
:102C400002F01AF8192360616376206121232020A5
:102C50000121A37684F8A20002F0E2FA1F230F20DC
:102C600084F8A830207102F007F8A06094F8A8005A
:102C700002F002F81C2384F824301B2384F825304A
:102C8000242384F82630252384F82730112384F860
:102C90002830132384F82930142384F82A3015238C
:102CA00084F82B30172384F82C30162384F82D3029
:102CB000122384F894301A23C4F8AC0084F89530B9
:102CC0001020012102F0ACFA2946102002F088FA07
:102CD0000E2084F8A100012102F0A2FA97E0052F4E
:102CE00040F091800223152084F8A03084F8BD00C4
:102CF000012102F095FA384684F8BE70012102F0F5
:102D00008FFA062084F8BF00012102F089FAFF2221
:102D10002B4620462946FFF760FD142060730121F1
:102D200002F07EFA1020A07301F0A6FF1923606163
:102D300063762061212320200121A37684F8A2005C
:102D400002F06EFA1F230F2084F8A830207101F0E2
:102D500093FFA06094F8A80001F08EFF1C2384F874
:102D600024301B2384F82530242384F8263025239F
:102D700084F82730112384F82830132384F829306D
:102D8000232384F82A30222384F82B30172384F855
:102D90002C30162384F82D301223C4F8AC0084F8AC
:102DA00094300E201A2384F8953084F8A100012174
:102DB00002F036FA0920012102F032FA29460920F0
:102DC00002F00EFA0B20012102F02AFA29460B200C
:102DD00002F006FA0C20012102F022FA29460C200A
:102DE00002F0FEF91D20012102F01AFA29461D20E9
:102DF00002F0F6F91E20012102F012FA1E202946E7
:102E000002F0EEF903E0FE23C4F8E4303CE0204693
:102E1000FFF7A4FD207901F02FFF237EA06043B1CE
:102E2000607E03F09FFBE061A07E03F09BFB2062CD
:102E300001E0E3612362237B83B1607B012102F027
:102E4000EFF9A07B01F018FF2061236907E000BFC4
:102E5000E39B000088F00F4048F00F40236163615E
:102E600004F10A062546002385F88A30A36595F803
:102E7000240085F880302F1B01F0FEFE0C37013551
:102E8000B54244F82700EED1204604B0BDE8F081F9
:102E900010B5D0F8E430032B044690F8A1000ED111
:102EA000012102F0BDF994F8A120084B53F832300B
:102EB000012283F88020642002F0D0FA02E0002191
:102EC00002F08EF9002384F8F53010BD38A9000017
:102ED00010B50446FFF7DCFF4FF4C87002F0BEFAED
:102EE0002046BDE81040FFF739BDFFFF014B024A05
:102EF0001A6070470CED00E00400FA052DE9F84F68
:102F00004FF0000891F803900B7982F8023182F8B3
:102F1000048109EB030A04461546FFF7FDFC0AF19C
:102F2000FF3A5FFA8AFA074609EB0803DBB253451A
:102F300000F200825FFA88F6B82B00F2F581DFE834
:102F400013F0B9001701BC00C000C400F301F30185
:102F5000F301F301F301F301F301F301F301F301D1
:102F6000F301C800F301F301F301CC00F301F30115
:102F7000F301F301F301F301F301F301F301F301B1
:102F8000F301F301F301F301F301F301F301F301A1
:102F9000F301F301F301D000D500F301F301F301D4
:102FA000F301F301F301F301F301F301F301F30181
:102FB000F301F301F301F301F301DD00F301E1009B
:102FC000E500E900ED00F100F500F9000601F3016C
:102FD0000C011701F3011001F30113011701F301B3
:102FE0001A01F3011D012501F3012101F30125015E
:102FF0003C0128012D0132013701F3014101440157
:103000004D01F301560159015E0163016801F301AD
:103010006D01730179018401F30190019201940122
:10302000960198019A019C019E01A001A201A401B0
:10303000A601A801AA01AC01AE01B001B201B40120
:10304000BA01F301C201C501C801CB01CE01D10112
:10305000D401D701DA01DD01F301F301F301F3013A
:10306000F301F301F301F301F301F301F301F301C0
:10307000F301F301F301F301F301F301F301F301B0
:10308000F301F301F301F301F301F301F301F301A0
:10309000F301F301F301F301F301F301F301E001A3
:1030A000F301E301F301E601F301E901F301EC01AE
:1030B000F301EF012E44952338E12046FFF70BFC86
:1030C000F7E02046FFF72EFCF3E02046FFF7BCFBBD
:1030D000EFE02046FFF7D4FBEBE02046FFF716FCBD
:1030E000E7E0D4F8AC0001F013F9E2E0A06801F0E9
:1030F00005F90A232E4490FBF3F0E2E02046FFF7A7
:10310000DEFBD6E02046FFF7E0FBD2E02046FFF7EB
:10311000DCFBD4E02046FFF7E7FBCAE02046FFF7E0
:10312000E9FBC6E02046FFF7EBFBC2E02E4494F833
:10313000F530FBE02046FFF77EFB83462046FFF795
:1031400077FB2BF00F032E4403EB2010B9E0204651
:10315000FFF774FB2E440011B3E02046FFF793FB0A
:10316000A7E02E44744B0FE02046FFF799FBA0E048
:103170002E440123DAE02E44704B05E02046FFF791
:1031800098FB96E06E4B2E441B78CFE02E44032331
:10319000CCE06C4B1868FDF7CFFD8AE0694B1868EE
:1031A000FDF7A6FD85E0674B1868FDF7C9FD80E0D7
:1031B000644B1868FDF7C4FD81E0634B1B6893F80E
:1031C000BC30AFE02E44237BB0E02046FFF79EFBEF
:1031D00062692369D31A23EAE37330E02046FFF7DC
:1031E00095FB62692369D31A23EAE37332E02E4424
:1031F000237E9BE02046FFF789FBE3691FE0204622
:10320000FFF784FBE36925E02046FFF77FFB236A95
:1032100015E02046FFF77AFB236A1BE02046FFF704
:1032200075FBD4F89C300AE02046FFF76FFBD4F81A
:103230009C300FE02046FFF769FBD4F8983008B1C6
:10324000DBB26FE0C3F387036CE02046FFF75EFB61
:10325000D4F8983010B1C3F3072363E0C3F3872396
:1032600060E0206B22E0206B26E0606B1EE0606B6C
:1032700022E0A06B1AE0A06B1EE0E06B16E0E06BB2
:103280001AE0206C12E0206C16E0606C0EE0606CBE
:1032900012E0A06C0AE0A06C0EE0E06C06E0E06CCE
:1032A0000AE0206D02E0206D06E0606D394601F015
:1032B00034F82E4405E0606D394601F02EF82E44B6
:1032C0000012F07033E094F88A302BE094F88B30E1
:1032D00028E094F88C3025E094F88D3022E094F8C2
:1032E0008E301FE094F88F301CE094F8903019E095
:1032F00094F8913016E094F8923013E094F89330FB
:1033000010E023681B780DE023685B780AE02368EF
:103310009B7807E02368DB7804E023681B7901E0F1
:1033200023685B792E4401E02E440023F37008F1FA
:103330000108F9E5BDE8F88FF490FF1FC388FF1F6F
:10334000F590FF1FAC88FF1FB488FF1F2DE9F74FD2
:10335000002782F8027191F803A091F802B182F877
:103360000471D344ABF1020B0546894616465FFA59
:103370008BFBB846FAB202EB0A03DBB201325B45C3
:10338000D2B200F212814A44822BD47800F0E48059
:103390003DD8442B00F0988015D8052B00F0038110
:1033A00009D8032B69D0042B40F0F780284621462A
:1033B000FFF74DFAF7E0142B73D0432B79D0102B85
:1033C00040F0EB8065E05A2B00F0948017D8572B23
:1033D00000F0A680592B00F08480452B40F0DD8062
:1033E0002846FFF725FA014628460191FFF723FA00
:1033F000230102460199284603F0F0036EE0802B7A
:1034000000F0A18000F2A5805B2B75D0C5E0892B70
:1034100000F0B18015D8852B00F0A48009D8832B4B
:1034200000F09D80842B08BF85F88D4000F0BB80A4
:10343000B3E0872B00F0998000F29A8085F88F40E6
:10344000B1E0B22B00F0A0800BD8AE2B00F096803C
:10345000B02B00F096808A2B40F09F8085F8934037
:10346000A1E0B62B00F09380B82B00F09380B42B32
:1034700040F093802B68DC7095E028462146FFF7EA
:1034800059FA002840F0898028462146FFF74DFA76
:1034900089E0022C00F2818028462146FFF7DDF901
:1034A00081E028460CB9214600E00021FFF751FADF
:1034B00079E01CB92846FFF7EBFC74E0012C6CD1D5
:1034C0002846FFF74BFA6EE02846FFF7B7F92101CF
:1034D000034601F0F001284604F0F002FFF77DF901
:1034E00061E0334B186814B9FDF712FC5BE0FDF79F
:1034F00001FC58E0A04656E008EB042142F20F73AD
:10350000994204DC2A4B1868FDF714FE05E096F892
:10351000043143F0080386F804314FF0000842E01C
:1035200014F0F00239D123462BB1D90744BF013240
:10353000D2B25B08F8E7022A00D074BB1D4B1B68AF
:1035400083F8BC402FE074B31B4B186800F03EFDBD
:1035500029E085F88A4026E085F88B4023E085F84D
:103560008C4020E085F88E401DE085F890401AE000
:1035700085F8914017E085F8924014E02B681C70A4
:1035800011E02B685C700EE02B689C700BE02B68E0
:103590001C7108E02B685C7105E096F8043143F07B
:1035A000080386F804310137E4E603B0BDE8F08F84
:1035B000AC88FF1FB488FF1FBC88FF1F38B5C56AE1
:1035C000094B036004462DB12846FFF7FDF8284655
:1035D00003F0F6FE206A04F0D3FB201DFDF72EFE5B
:1035E000024B2360204638BD089C0000B08C0000D0
:1035F00010B50446FFF7E2FF204603F0E1FE204647
:1036000010BDFFFF2DE9FF4106461A4B46F8043B6B
:103610000446002530460F469046FDF7E1FD84F84C
:10362000305084F8395184F83F522577FF2004F058
:103630009FFB206250B91049684603F0A5FF684619
:1036400000F0B6FE684603F05FFF0FE030464146EB
:10365000FDF7EAFDA7610C2003F0B0FE0646FFF778
:103660006AF80123E66284F830502377204604B0DC
:10367000BDE8F081089C0000EF9B000038B50446CF
:10368000806903689B689847E8B1251D2846FDF7C7
:1036900039FEA06903689B68984718B12846FDF772
:1036A0000DFE38B194F830301BB1074B1B68A36294
:1036B00038BD38BDA0690368DB689847C1B22846A9
:1036C000FDF7C6FDE5E738BDF488FF1F70B588B08B
:1036D00004460E46069300219DF8303007934FF4C0
:1036E00083708DF815108DF8142004F041FB3146DD
:1036F0004FF48372054601F003F96B4643F8044B1F
:1037000008AC14E9070083E80700044B2946186851
:1037100001221E2300F08AFB08B070BDBC88FF1F89
:1037200007B500230093FFF7D1FF03B05DF804FB5A
:1037300070B588B000244FF483700E468DF81540A4
:10374000069404F015FB31464FF48372054601F0F0
:10375000D7F86B4608AE43F8044B16E9070083E838
:103760000700044B294618682246234600F05EFBFA
:1037700008B070BDBC88FF1F10B50446E06AFEF7B4
:10378000DFFF00280ADDE06AFFF700F8406808B1B3
:1037900004F0F6FAE06AFFF71DF8EFE7002384F87B
:1037A000303010BD38B591F802314C781C440B789C
:1037B00002340A2B0D46E4B201D18B7803E0142BBE
:1037C00004D191F804311C44E4B202E00E2000F070
:1037D000ABFD95F802210023934205DAE918013385
:1037E000C9780C44E4B2F7E7E043C0B238BD83299E
:1037F00006D003D80139022904D801E0922901D169
:10380000012070470020704738B50346006AFF2248
:103810000270186A42701A6A4878907091F8020132
:103820001A6A0230D0701A6A91F8040110710020EF
:1038300091F80251C4B2621DA542D2B21C6A08D9E5
:10384000FA2805D00A180444D27862710130EFE7F3
:10385000FD2291F80311A1549869016801324C6866
:10386000196AD2B2A04738BD70B5142380F83A3136
:103870008B780022013B04460D4680F83E22052B42
:1038800027D8DFE803F003091426261F6B7880F899
:103890003B3180F83C221CE06B7880F83B31204BB8
:1038A0002946186804F59D72FFF728FB11E06B7834
:1038B00080F83B311A4B2946186804F59D72FFF7D2
:1038C00045FD06E0164E3068FFF7E2FA3068FFF774
:1038D0000DFB94F83B31FE2B20D095F80531EBB968
:1038E0000F4E3068FEF7CCFF022809D03068FEF793
:1038F000C7FF0128AB7801D1022B01D0012B0DD1DC
:1039000004F59D7529462046FFF74CFF84F83D02DB
:1039100029462046BDE87040FFF776BF70BD00BF66
:10392000B488FF1F2DE9F04F85B0CA7891F804B034
:10393000039207460D46022495F80231A3423DD971
:10394000204E05EB0409306899F803A0FEF7EAFF62
:1039500082450BF1010804D030685146FEF7EAFFBA
:10396000C8B14B46039A03F8032F5FFA88F200921E
:10397000154A03211068524600F09DFA81463068CE
:10398000FEF7D0FF824509D1012389F80531384679
:103990004946FFF769FF4444E4B2CDE7094B51467D
:1039A0001868FEF7C7FF28B1384649460222FFF7DC
:1039B000B7FEF0E7122000F0B7FCECE705B0BDE879
:1039C000F08F00BFB488FF1FBC88FF1FF8B5044606
:1039D000E06AFEF7B5FE002804DC2046BDE8F840AA
:1039E000FFF7CABEE06A184FFEF7D0FE057806461C
:1039F0003868FEF797FF85427168204602D1FFF7CD
:103A000033FF02E00322FFF78BFE706804F0B8F981
:103A1000E06AFEF7DFFE0D4B38681B68A362FEF715
:103A200081FF85420FD1E06AFEF78AFE002806DD9D
:103A3000E06AFEF7ABFE4378AB42C9D0F8BD94F81C
:103A40002530AB42C9D0F8BDB488FF1FF488FF1FF2
:103A500070B5012380F830300B4B0C4D1B6890F88B
:103A60002460836204462868FEF75CFF864205D026
:103A7000286894F82410FEF75DFF20B12046BDE8C9
:103A80007040FFF7A3BF70BDF488FF1FB488FF1F0D
:103A90002DE9F0434B7980F8243091F802310B4442
:103AA00085B05B7880F8253006460C4601254FF03E
:103AB000FF0994F80231AB4215D96F1CDFF874800E
:103AC0002744D8F80000F978FEF734FF88B9D8F811
:103AD0000000FEF727FFFB7883420AD0033597F8F2
:103AE0000390EDB2E5E73046FFF7B2FF05B0BDE861
:103AF000F0830821012004F00BF9FA7802706319B1
:103B000080F801905979DB788DF80C108DF80D3024
:103B10000221074B00918046186803AB00F0CBF9F7
:103B20004146C8F80400F06AFEF70CFED6E700BF75
:103B3000BC88FF1FB488FF1F2DE9F843037F0446AC
:103B4000002B00F0CC8090F830302BB1654B1A6818
:103B5000836AD31A642B19D82046FFF78FFD251DE1
:103B60002846FDF78BFB05280EDD28460021FDF7D2
:103B70008FFBFF2840F0AB8028460121FDF788FB32
:103B8000FF2840F0A48004E0BDE8F883FFF7F4FDCF
:103B9000E2E702212846FDF77BFB002384F835008D
:103BA00084F8393128460321FDF772FB01280746C6
:103BB00007DD2846FDF762FBFE1C864203DBBDE8FD
:103BC000F883BDE8F88394F830304BB1142384F8BF
:103BD000343028460421FDF75BFB84F8380108E007
:103BE0000A2384F8343028460421FDF751FB84F879
:103BF0003600BB1E5FFA86F884F836310526F3B22C
:103C00004345284607D23146FDF742FBA31901364A
:103C100083F83200F3E74146FDF73AFB04F134063E
:103C200084F8370131462046FFF7BCFD94F8373160
:103C300083424CD194F830309BB1E06AFEF7A6FD88
:103C400094F8353042789A4203D12046FFF7BEFE01
:103C500040E094F825209A423CD12046FFF78CFDA5
:103C600038E0204694F83610FFF7C1FD90B3DFF836
:103C7000788094F83590D8F80000FEF753FE81451F
:103C800020D0D8F8000094F83510FEF753FE28B184
:103C9000204631460122FFF743FD1BE094F8353002
:103CA000FE2B17D194F83630832B2046314602D1B3
:103CB000FFF738FE0EE0922B02D1FFF7E9FE09E094
:103CC000FFF736FD20463146FFF7CEFD02E02846DD
:103CD000012101E02846391DFDF7FEFA3FE7BDE866
:103CE000F88300BFF488FF1FB488FF1F30B585B08C
:103CF00004AC04E90E00089C9DF804300546002C35
:103D000035D0012B03D12146FFF77EFD21E0032BA7
:103D100025D190F83030A3B12146FFF775FD154B42
:103D2000E86A1B68AB62FEF70BFD002809DDE86A54
:103D3000FEF72CFD637842789A4202D12846FFF7BD
:103D400045FE627895F825309A4202D12846FFF761
:103D500013FD204605B0BDE8304004F011B8022B39
:103D600005D0132005B0BDE8304000F0DDBA05B045
:103D700030BD00BFF488FF1F38B58568154B036060
:103D800004462DB12846FDF759FA284603F018FBE2
:103D9000A069FEF7D5FC00280FDDA069FEF7F6FC50
:103DA000C06803F0EDFFA069FEF7F0FC406803F087
:103DB000E7FFA069FEF70EFDEAE7A5692DB12846E9
:103DC000FEF702FD284603F0FBFA034B2360204672
:103DD00038BD00BF209C0000B08C000010B5044628
:103DE000FFF7CAFF204603F0EBFA204610BDFFFFA5
:103DF0000D4B70B503600446C1601420164603F0F5
:103E0000DDFA0546FDF7ECF93146A5602846FDF7D9
:103E10000BFA0C2003F0D2FA0546FEF78CFC0023C7
:103E2000A5612374204670BD209C00002DE9F04759
:103E300008AE07460D4601201821904656F804ABFF
:103E4000994603F065FF45600446054696E807007D
:103E500045F808AB85E8070084F8159084F81480CD
:103E6000B8692146BDE8F047FEF76CBC38B591F85B
:103E700002314C781C440B7802340A2B0D46E4B214
:103E800001D18B7803E0142B04D191F804311C4448
:103E9000E4B202E00B2000F047FA95F8022100237B
:103EA000934205DAE9180133C9780C44E4B2F7E724
:103EB000E043C0B238BD2DE9F8430F4606464FF443
:103EC00083710120904699469DF8205003F020FF11
:103ED0000A230446037080F8018087700022D3B261
:103EE000AB4205D2A31819F80210D9700132F6E7D7
:103EF00084F8025130462146FFF7B8FF84F80301E9
:103F00002046BDE8F883FFFF2DE9F0418CB006465E
:103F100005A880E80E009DF81430129D069C012B28
:103F200045D1079B022B02D0032000F0FDF955B1CB
:103F30002378092B07D8244A11685A1C22700B4495
:103F40006A7883F88A206378FC2B04D894F8008080
:103F5000B8F1090F03D9204603F012FF2AE002202E
:103F600003F006FF80F8008062780132002301240C
:103F7000D2B20221427007460B910093214630468F
:103F80008DF825308DF82440FFF795FF6B460A9792
:103F900043F8046B0CAF864617E9070083E8070077
:103FA0003046714622460623FFF740FF02E0042018
:103FB00000F0BAF92DB128460CB0BDE8F04103F08D
:103FC000DFBE0CB0BDE8F081B488FF1FF0B5194B1F
:103FD00089B0196806460023CA18013300250A2B48
:103FE00082F88A50F8D102208DF8155003F0C0FEF7
:103FF00001240570447007460095214622462B4651
:1040000030468DF81440FFF756FF022307936B46A6
:10401000069743F8046B08AF054617E9070083E8E5
:1040200007003046294622460623FFF7FFFE09B067
:10403000F0BD00BFB488FF1FF0B589B005238DF82F
:104040001030022300240093032104ABFE22054616
:104050008DF8154006948DF81140FFF72CFF6B4644
:1040600008AF43F8044B064617E9070083E807004A
:104070002846314622462346FFF7D8FE09B0F0BD58
:104080002DE9F04104468068FDF7F8F801283CDD91
:10409000A0680021FDF7FCF8FF2805D1A0680121E8
:1040A000FDF7F6F8FF2804D0A0680121FDF714F908
:1040B0002BE0A068FDF7E2F8052826DD0221A068C4
:1040C000FDF7E6F803210646A068FDF7E1F80128B0
:1040D00007461AD9A068FDF7D1F807F10308804513
:1040E00016DB12E04146FDF7D3F82946064685F86F
:1040F00003012046FFF7BAFE8642A06829D00121BD
:10410000FDF7EAF8284603F03BFE0020BDE8F08109
:104110004FF48371012003F0FBFD14234670054624
:1041200003700421A068FDF7B3F8BB1E85F80401F5
:1041300085F802315FFA88F80526F3B24345A06896
:10414000D0D23146FDF7A4F8AB19013603F8020CC2
:10415000F3E7391DFDF7C0F82846BDE8F08170B5DA
:104160000546C0680A230B7003680C461B68FF21D4
:104170009847E8680368FF211B689847E8686178FA
:1041800003681B689847E86894F8021103680231D5
:104190001B68C9B29847E868A17803681B6898470C
:1041A000002394F80221E8685E1CDBB29A4206D92B
:1041B00023440268D978126890473346F1E70368D0
:1041C00094F803111B68984770BDFFFF73B5044650
:1041D000E06803689B68984758B1E0680368DB684B
:1041E0009847C1B2A068FDF733F8354B1B6863618F
:1041F000EEE7237C4BBBA069FEF7A2FA00285CDD4A
:10420000A068FDF765F8A069FEF7C0FA05462046EC
:104210006968FFF7A4FF6B685B78FE2B06D1062068
:1042200001F01CF920466968FFF799FF2B7D237484
:1042300043B9E86803F0A4FD686803F0A1FDA06934
:10424000FEF7C8FA1E4B1B681AE0012B1AD1A069B1
:104250001B4EFEF79BFA05462046FFF711FF32681A
:104260006369A8B9697DD31A8B4226D96B7A012B71
:104270000ED801336B7220466968FFF770FF336810
:1042800063611AE00C2002B0BDE8704000F04CB849
:104290002B683BB11A680090184605F108031668B0
:1042A0000ECBB047E86803F06BFD686803F068FD6B
:1042B000A069FEF78FFA0023237402B070BD00BF1F
:1042C000F488FF1FFB280CD0FC2803D0FA2803D168
:1042D0000548704705487047054B0130B3FBF0F0C7
:1042E00070470448704700BF10552200C0C62D001B
:1042F00080841E00A0252600400070478010EE3804
:10430000024B20EAE07053F820007047309C000018
:1043100040F26B135843000B704740F2DE73584372
:10432000B0FBF1F07047FFFF70B505462C46002C3E
:1043300023DD012D12DD134E306878B100221346C3
:10434000FF21FEF74AFA4FF47A7001F087F8002156
:1043500030680A460B46FEF740FA08E00A4B202672
:104360001E604FF47A7001F079F8084B1E604FF42C
:104370007A7001F073F8013CD9E74FF47A6001F0EC
:104380006DF8D3E7B488FF1F84F00F4088F00F402A
:10439000054B1A6840F6B7339A42014602D90348E2
:1043A00003F010B8704700BFF488FF1FD890FF1FBC
:1043B00008B5084B1A6840F6B7339A42014607D948
:1043C000054802F0FFFF0448BDE8084003F01AB8B2
:1043D00008BD00BFF488FF1FD890FF1F08B5084B29
:1043E0001A6840F6B7339A42014607D9054803F0E8
:1043F00064F80448BDE8084003F004B808BD00BFF5
:10440000F488FF1FD890FF1F072910B50C460BD862
:1044100072B600F08BFD62B60123A3401840C0B213
:1044200040FA04F4E0B210BD002010BD08B572B629
:1044300000F07CFD62B608BD08B572B600F08AFDDA
:1044400062B608BD2DE9FF41234D2B68642B07465A
:104450000C4690462E460DDD2049684603F094F840
:104460006846FFF795FF684603F04EF82868FFF7A7
:10447000B5FF2DE0072921D800F080FD0028FBD0F2
:1044800072B6384600F052FD62B6012303FA04F416
:1044900018F0010F0CBF20EA04040443E4B200F05A
:1044A0006DFD0028FBD072B63846214600F06EFD47
:1044B00062B633680133336001200AE00849684678
:1044C00003F062F86846FFF773FF684603F01CF8D4
:1044D000002004B0BDE8F081C488FF1F40A80000A0
:1044E00095A8000070B50B4C2368642B05460E465A
:1044F0000EDC00F043FD0028FBD072B628463146A2
:1045000000F044FD62B6236801332360012070BDD2
:10451000002070BDC488FF1F70B50B4C2368642B4E
:1045200005460E460EDC00F029FD0028FBD072B6D1
:104530002846B1B200F044FD62B62368023323601E
:10454000012070BD002070BDC488FF1F10B5044657
:1045500059B101210B20FFF7C5FF00210C20FFF707
:10456000C1FF0D200221FFF7BDFF631EDBB2FC2B54
:1045700005D821460E20BDE81040FFF7B3BF10BD9F
:1045800008B500210220FFF7C7FF00211720FFF721
:10459000C3FF002101221720FFF754FF01210A4623
:1045A0001720FFF74FFF41F244611A20FFF7B4FFD5
:1045B00003210F20FFF796FF10200146FFF792FF1F
:1045C00001211320FFF78EFF01211420FFF78AFF3E
:1045D00003211520FFF786FF03211620FFF782FF36
:1045E00001200146BDE80840FFF7B0BF084B1A683C
:1045F00042F480721A604FF4A072013A7FF4FDAF6A
:104600001A689205FCD42023013B7FF4FDAF70476C
:10461000005004402DE9F74F6A4E6B4B3268517ED3
:10462000927E5C5C9D5CFF2C814601D0FF2D02D107
:104630001120FFF779FE3168644A4B7E644F02EB2C
:10464000C303586800230360897E624802EBC102FD
:10465000614952681360614B620013440B605F4B09
:104660006A0013443B605E4B1A6842F020021A60F5
:1046700001235C4A03FA05F503FA04F445EA04034E
:104680001360594B1A6822F080021A60574A106072
:10469000574818608846B9F1000F7AD0142000F00E
:1046A000DDFEFFF7A3FFD8F8003052491B889BB20C
:1046B000ADF80030BDF80030BDF800204E4B92B28E
:1046C0000A601A603A684D49128892B2ADF8022029
:1046D000BDF80220BDF8022092B20A6048494FF0AE
:1046E0000A0A0A609946FFF781FFD8F80030414D69
:1046F0001B88D9F800203868404C9BB2ADF80430D4
:10470000BDF80430BDF804103E4B89B219602B6827
:104710004FF0060B42F20F7E0BFB02120EFB03134F
:1047200042F21071B3FBF1F32B6003889BB24FF0A0
:10473000070CADF80630B2FBFCF2BDF80630BDF850
:104740000600C9F8002022682F4B80B20BFB020242
:10475000DFF8ACB01860DBF800300EFB0303B2FBEF
:10476000FCF2B3FBF1F105200AF1FF3A2260CBF82D
:10477000001000F073FE1AF0FF0AB4D11E4A33682D
:1047800011682A688A1ADA612168DBF800208A1A1F
:104790001A62154B15491A6822F080021A600A68DD
:1047A00042F420620A601A6842F0D2021A60174B83
:1047B00080221A70A3F24B334FF400221A6003B028
:1047C000BDE8F08FB488FF1FECA8000038A90000F6
:1047D000E488FF1F00000303E088FF1F005104402E
:1047E0003880044008500440005004400450044005
:1047F00080004D00E888FF1FDC88FF1FD488FF1F62
:10480000C888FF1FD888FF1FD088FF1F53E400E02F
:104810002C4BF7B51A6812F4805F1A680AD042F47C
:1048200080521A60284B1A68002001321A60FFF784
:10483000F1FE45E042F400421A60244B1B681B88DD
:104840009BB2ADF80430BDF80430BDF80420204B15
:1048500092B21A601F4B1C684FF0060C07270CFB26
:104860000424B4FBF7F41C601B4B196842F20F766A
:1048700006FB012242F21075B2FBF5F21A60174BEB
:1048800017491B681B889BB2ADF80630BDF806308F
:10489000BDF806309BB20B60124908680CFB003073
:1048A000B0FBF7F0086010490F6806FB0733B3FB55
:1048B000F5F30B600D490968A21AC31ACA610B62AD
:1048C00003B0F0BD00500440CC88FF1FE088FF1FFC
:1048D000D888FF1FDC88FF1FE888FF1FE488FF1FC0
:1048E000D088FF1FD488FF1FC888FF1FB488FF1F10
:1048F000024B4FF400221A60704700BF88E100E0CD
:10490000844641EA000313F003036DD1403A41D3DA
:1049100051F8043B40F8043B51F8043B40F8043B99
:1049200051F8043B40F8043B51F8043B40F8043B89
:1049300051F8043B40F8043B51F8043B40F8043B79
:1049400051F8043B40F8043B51F8043B40F8043B69
:1049500051F8043B40F8043B51F8043B40F8043B59
:1049600051F8043B40F8043B51F8043B40F8043B49
:1049700051F8043B40F8043B51F8043B40F8043B39
:1049800051F8043B40F8043B51F8043B40F8043B29
:10499000403ABDD2303211D351F8043B40F8043BC9
:1049A00051F8043B40F8043B51F8043B40F8043B09
:1049B00051F8043B40F8043B103AEDD20C3205D3D9
:1049C00051F8043B40F8043B043AF9D2043208D0D1
:1049D000D2071CBF11F8013B00F8013B01D30B8843
:1049E00003806046704700BF082A13D38B078DD021
:1049F00010F003038AD0C3F10403D21ADB071CBFF3
:104A000011F8013B00F8013B80D331F8023B20F85C
:104A1000023B7BE7043AD9D3013A11F8013B00F895
:104A2000013BF9D20B7803704B7843708B7883701D
:104A300060467047F0B5304B1B681B06FBD42F4B0C
:104A40001B6813F08002F6D172B62D4B197800293D
:104A500050D02C4908684F688E68CD680C6938447E
:104A6000143130440968284420440844C0F34E00FF
:104A7000254940F400400860C86A0F6B4E6B8D6B8F
:104A8000CC6B384440313044096828442044084401
:104A9000C0F34E001D4940F40040086001F10811C8
:104AA000143151F8140C51F8107C51F80C6C51F879
:104AB000085C51F8044C09683844304428442044C8
:104AC0000844C0F34E00124940F400400860C86A30
:104AD0000F6B4E6B8D6BCC6B3844403130440968A2
:104AE000284420440844C0F34E000A4940F40040E2
:104AF00008601A7062B6F0BD24B0034024B00B40C9
:104B0000ED88FF1F38B003402CB0034030B00340A5
:104B10002CB00B4030B00B4010B5204B2048214941
:104B200060221A70E1225A701F4B204A1C78204BD9
:104B3000082C01D1012402E00A2C03D1392404609D
:104B4000132005E00C2C0CBF35243D2404601220FA
:104B5000086014601860174B17491B78174A03B197
:104B600001230B601360164B164A1978164B012966
:104B700001D880210BE0042901D8842107E008290D
:104B800001D8852103E0102994BF86218721116077
:104B900019600E4B01221A7010BD00BF0040074083
:104BA00008B003400CB003406487FF1F08B00B40FF
:104BB0000CB00B40F088FF1F20B0034020B00B402A
:104BC0006587FF1F24B0034024B00B40ED88FF1F12
:104BD0000C2804D9102828BF1020102307E00A2829
:104BE00004D8092834BF08230A2300E00C23094A0B
:104BF000D9B2081A1070084A1078834208D0074BBF
:104C000011701B7813B1064B00221A60FFF784BFA6
:104C1000704700BFEC88FF1F6487FF1FED88FF1FF0
:104C200024B0034010B5114B1B7804460BB1FFF7BD
:104C300001FF012C0E4A01D8002302E0042C02D807
:104C4000042313600EE0082C03D805231360082307
:104C500008E0102C03D806231360102302E007237A
:104C600013602023034A137010BD00BFED88FF1F9F
:104C700024B003406587FF1F0D2838B50FD91728CA
:104C800001D80E380AE0A0F11A03052B01D8093823
:104C900004E0A0F12203062B47D81838C0B2244BF9
:104CA0001C5C244B1B780BB1FFF7C4FE210614D407
:104CB00072B6214B214D1C6001232B7062B672B677
:104CC0001D4B1B681A0601D51D4B1FE02B78002BCE
:104CD000EFD062B602F084FCF1E772B6194B1A4DC0
:104CE0001A6814F0400F14BF22F0100242F01002B4
:104CF0001A60164B04F03F021A6001232B7062B653
:104D000072B6124B1B681B0608D5114B186800239E
:104D10002B7062B60F4B1B78184138BD2B78002BD7
:104D2000DCD062B602F05CFCEAE7002038BD00BFD0
:104D30000EA90000ED88FF1F00B00340EF88FF1FA1
:104D400010B003400CB00B40EE88FF1F00B00B40CA
:104D500010B00B40EC88FF1F0D2810B50FD9172895
:104D600001D80E380AE0A0F11A03052B01D8093842
:104D700004E0A0F12203062B27D81838C0B2134B49
:104D80001C5C134B1B780BB1FFF754FE230607D4B2
:104D900072B6104B44F040041C6001220E4B12E02E
:104DA00072B60E4B1A6814F0400F14BF22F01002B6
:104DB00042F010021A6004F03F04094B44F0400432
:104DC0001C60084B01221A7062B610BD0EA90000CB
:104DD000ED88FF1F00B00340EF88FF1F0CB00B40B1
:104DE00000B00B40EE88FF1F0D280FD9172801D8FF
:104DF0000E380AE0A0F11A03052B01D8093804E0A7
:104E0000A0F12203062B26D81838C0B2134B1B562C
:104E1000002B08DB124B1B6813F0800F114B12D0D4
:104E200072B6114A07E0114B1B6813F0800F104B4C
:104E300009D072B60F4A106800221A7062B60E4B83
:104E40001B78184170471B78002B14BF4FF0FF30C0
:104E50006FF0010070470020704700BF0EA90000EE
:104E600000B00340EF88FF1F10B0034000B00B40BC
:104E7000EE88FF1F10B00B40EC88FF1F084B1A682C
:104E800042F480521A60074B1A78074B0AB180220D
:104E900000E0C0221A70054B80F30C0018807047A8
:104EA0002C800440F088FF1F21C00C4000C00C4043
:104EB000024B1B78DB07FBD5704700BF01000240A7
:104EC0007FB5174B6A4603F110056E46186859689E
:104ED000144603C40833AB422246F7D1114B1A786B
:104EE00012F0020F1D4612D080229A7133229A725C
:104EF00003225A7272B60C4C46F001062046B047A7
:104F000062B6237813F0700301D0237006E044F6F4
:104F100021632A78D20701D4013BFAD104B070BDD5
:104F200026A900000100024000000240B0F5006F19
:104F300010B5044609D2064B1B78DB0701D4FFF7F6
:104F4000BFFF04F1A054207810BD002010BD00BFA9
:104F50000100024040F2FE73984210B5044609D8A1
:104F6000054B1B78DB0701D4FFF7AAFF04F1A0541F
:104F7000208810BD002010BD01000240024B1878AF
:104F800000F00100704700BF01000240B0F5006F63
:104F900038B504460D460FD2084B1B78DB0701D409
:104FA000FFF78EFF04F1A0542378AB4204D02570A4
:104FB000BDE83840FFF77CBF38BD00BF01000240AC
:104FC00038B540F2FE73984204460D461ED8104B89
:104FD0001B78DB0701D4FFF773FF14F0010F04F116
:104FE000A05404D12388AB4210D025800AE0237856
:104FF000AB4202D02570FFF75BFF63782D0AAB420E
:1050000004D06570BDE83840FFF752BF38BD00BF1F
:1050100001000240024B1A6801321A60704700BF5B
:10502000F488FF1F08B50B4C2368580301D501F025
:10503000A3FB2368590501D500F0CAFC23681A05B3
:1050400001D500F0A7FF2368DB04ECD501F010FACE
:10505000E9E700BF3480044008B5FFF7E3FFFFFF36
:10506000014B10221A807047002005407047FFFF57
:10507000024A136818441060184670476887FF1F7B
:10508000002070474FF0FF3070474FF0FF307047FF
:10509000FEE7FFFFEFF313839BB9EFF3108098B99E
:1050A000EFF3058323B10F2B04D9084A985C01E084
:1050B0004FF48070EFF311833BB1834238BF184641
:1050C00070474FF0FF30704718467047F0E300E03C
:1050D000044B054900221A600A60044A106010223D
:1050E0001A60704714D0034004D0034000D003403E
:1050F0002DE9F04105460E4608462E4902F092FD84
:105100002D4B002847F6122814BF0227012708BF9D
:105110009846002428FA04F002F08EFB4FF05E510E
:1051200002F0E2FB0146304602F090FD10B9013476
:10513000072CEFD128FA04F002F07EFB314602F092
:1051400087FC4FF07C5102F0C5FA02F0B9FD4FF632
:10515000FF73984228BF1846EB1E012B06D8174B49
:10516000174900221A600A60164A1BE0A5F10903DC
:10517000012B06D9A5F11403032B02D96B1F012BB8
:1051800006D8114B114900221A600A60104A09E042
:10519000202D01D0192D0BD10E4B0F4900221A6082
:1051A0000A600E4A04F0070444EAC70710601F6053
:1051B000BDE8F081001BB740006CDC0200900340AA
:1051C00004900340089003400080034004800340A3
:1051D0000880034000800B4004800B4008800B4097
:1051E000212810B518D80D4A52F8303093F8804273
:1051F0003CB1012211B183F8802010BD83F8002159
:1052000010BD02EBC00043681A6811B142F00302FE
:1052100001E022F002021A6010BD00BF38A90000B0
:10522000212816D80B4A02EBC00301295B6852F80B
:10523000302004D182F880124FF4A27208E00020DE
:1052400082F8800211B94FF4807201E040F203123B
:105250001A60704738A90000282838B5604A04460B
:105260000B4611D112780B2A04D8C2F10C0201FAB4
:1052700002F304E00C2A1CBF0C3A41FA02F3184670
:10528000BDE83840FFF7FABD11780125002B05FA7B
:1052900001F2D8BF002102DD934205D32946FFF772
:1052A0009FFF2046294697E00338C2B2012A01D861
:1052B0004C4A06E0202C01D0192C01D14A4A00E0CA
:1052C0004A4A126802FB0332CA401D287BD8DFE835
:1052D00000F0575F4E337A7A212A7A7A7A7A7A7A8C
:1052E0007A7A7A3C450F187A707A7A7A7A7A7A677B
:1052F0003F4B1A6003F5973340F2444203F5FA73CB
:105300005FE03C4B1A6003F5973340F2444203F5EB
:10531000F87356E0384B1A6003F5973340F2444275
:1053200003F5F6734DE0354B1A6003F5973340F201
:10533000444203F5F47344E0314B1A6003F59F33A4
:1053400040F2444203F5F0733BE02E4B1A6003F544
:105350009F3340F2444203F5EE7332E02A4B1A6069
:1053600003F59F3340F2444203F5EC7329E0274BE9
:105370001A6003F59F3340F2444203F5EA7320E0DC
:10538000234B1A6003F580334FF45172203318E039
:10539000204B1A6003F580334FF451721C3310E038
:1053A0001D4B1A60A3F5DB234FF45172A3F5F9638B
:1053B00007E01A4B1A60A3F5DB234FF45172A3F2F6
:1053C000CC731A6038BD7F2B2046D4BF0021012149
:1053D000FFF706FF20460121BDE83840FFF720BF58
:1053E0006C87FF1F0890034008800B400880034033
:1053F0001080034018800340208003402880034031
:1054000030800340388003404080034048800340A0
:10541000109003401890034010800B4018800B4000
:1054200072B60B4B0B491A680B4B1B68096862B6C6
:10543000490102D5322A88BF0133C2F5BB3260214F
:10544000FF32B2FBF1F24FF47A7000FB0320704799
:1054500018E000E004ED00E0F488FF1F38B50446D2
:10546000FFF7DEFF054624B938BD013C0AD005F53B
:105470007A75FFF7D5FF401BB0F57A7FF5D202F0C1
:10548000AFF8F6E738BDFFFF1F4B4FF4000210B531
:105490001A604FF080721A604FF000721A604FF07D
:1054A00080621A604FF000621A60184B184A194C5B
:1054B00000204BF6FF711860596028231360936039
:1054C00013619361136293621363936309222260F1
:1054D00004F58054043420606160A360236144F8C3
:1054E000042C04F5FE2420600B4801600B490B607E
:1054F0008B600B4B1A60FFF70FFBFA20FFF7AEFF34
:10550000BDE8104001F036BC08E100E00480034033
:105510000C8003400080034008800B400C800B404F
:1055200000800B401D4B1A6842F480621A601C4ACE
:10553000002313801B4A13801B4A13701B4A1370ED
:105540001B4A13701B4B40F213321A604FF4517216
:105550005A60194BC0F344321A70C0F347125A70A4
:105560000221042200F01F0098729A70D9745A75B3
:1055700088221A743C22DA709A7842F0A0029A705B
:105580009A7902F0DF029A710C4B40226FF44A7153
:105590001A700B444FF400521A6070473480044074
:1055A000808AFF1FFE88FF1F888AFF1F828AFF1FD5
:1055B000FC88FF1F40A0044000A006402DE400E04E
:1055C000134A937800F0030103F0EC030B43410707
:1055D00048BF43F01003937000F00F03042B0C49F5
:1055E00003D18B7943F040038B715379C20603F0EA
:1055F000EF03074A48BF43F01003537193798106C4
:1056000003F0EF0348BF43F010039371704700BFEE
:1056100000A0064008B5114B1B685B0500D408BD0F
:105620000F4B1A7802F0FF0312B101F0D9FFF7E730
:105630000C4A4FF4005111600B4A0C49D37040F2F0
:1056400003120A604A600A4A13800A4A13800A4B0E
:105650001B680BB101221A7008BD00BF34800440E2
:10566000FC88FF1F84E100E000A0064040A0044049
:10567000808AFF1FFE88FF1FF888FF1F38B5044689
:10568000094B1B7803F0FF05002BF9D120460121BF
:10569000FFF7C6FD20462946FFF7A2FD034B53F84E
:1056A0003420034B1A6038BDFC88FF1F38A9000066
:1056B000848AFF1F0D4A38B5146814F480624FF0D5
:1056C000000410D021280A4D0AD80A4A012152F8B4
:1056D00030302B60FFF7A4FD2B681C70012038BD13
:1056E0002C60204638BD104638BD00BF34800440D1
:1056F000F888FF1F38A900000E4B1B6813F4806365
:1057000016D012280C4B03D140F202310B4A04E0B0
:10571000142809D10A4A40F2023111605A7B42F042
:1057200001025A73012070475A7B02F0FE025A733D
:10573000002070473480044000A006400CA00440C4
:1057400014C00440F8B51F4B1B685A05064638D5EF
:105750001D4B1B680BB101221A701C4B9A7942F049
:1057600020029A711A4B1C780134802C1F4628BFE6
:105770000024184D2B78A34218D1FFF78BFC40284A
:105780000FDC124A13791B06F3D52B78124901332B
:10579000802B28BF0023C95CDBB2C9B2D1712B704A
:1057A000E7E7FF28E5DD01F01BFFE2E70A4BF6B271
:1057B0001E550A4B01221A70044BE4B2BC223C7005
:1057C000DA70F8BD34800440848AFF1F00A00640D0
:1057D000888AFF1F828AFF1F0089FF1FFC88FF1F26
:1057E000294B1B685A052DE9F04707468A4649D5DB
:1057F000264B1B680BB101221A70254B9A7942F097
:1058000020029A713D4607EB0A039D4237D2DFF82A
:105810009080204E98F8004096F800900134802C3B
:1058200028BF00245FFA89F9A1451DD1184BBC227D
:10583000DA70FFF72FFC40280FDC154A13791B069E
:105840000FD5337814490133802B28BF0023C95C5E
:10585000DBB2C9B2D171337003E0FF2801DD01F082
:10586000BFFE33784B45E4D00B4B15F8012B1A558E
:105870000A4B0122E4B21A7088F80040C3E7044BD7
:10588000BC22DA70BDE8F08734800440848AFF1FB0
:1058900000A00640828AFF1F0089FF1FFC88FF1FAF
:1058A000888AFF1F08B5034B1B7813B101F098FEDF
:1058B000F9E708BDFC88FF1F064A074B1B781078E4
:1058C000DBB2C0B283422CBF7F3000F1FF30C01A80
:1058D000704700BF828AFF1F888AFF1F054B188808
:1058E000054B1B8880B29BB2984238BF00F5807090
:1058F000C01A7047808AFF1FFE88FF1F114B124994
:105900001A880B8892B29BB29A4210B516D0013316
:10591000B3F5807F28BF00230C489CB2C05C0C808C
:105920000B490968C0B259B19A4238BF02F580727A
:10593000D31A1A2B04DC00230B7010BD4FF0FF307C
:1059400010BD00BF808AFF1FFE88FF1F8089FF1FD8
:10595000F888FF1F094B1A88094B1B8892B29BB22B
:105960009A4208D00133B3F5807F28BF0023054A4F
:10597000D05CC0B270474FF0FF307047808AFF1F85
:10598000FE88FF1F8089FF1F0C4B1B685B0514D529
:105990000B4BDA7802F0CB02DA7040225A74DA78D4
:1059A00042F03402DA70074B1A88074B92B21A8021
:1059B000064B1B680BB100221A70704734800440FC
:1059C00000A00640FE88FF1F808AFF1FF888FF1F87
:1059D00030B53E4B1A7912F0300F32D072B69A7D44
:1059E00002F0FF0022B9DA7940225A7462B628E048
:1059F00062B6374A3749138809889BB289B2144680
:105A0000324AD5795A1CB2F5807F28BF00228A42DB
:105A1000EDB202D0304B9D541346421E12F0FF00EF
:105A2000EED19AB222802D4A126852B18B4236BF13
:105A3000C1F58071C1EB03035B18272BC4BF0123A1
:105A40001370224BD978C9B20A0620D51B791D06DE
:105A50001DD5234B234A1D781378EDB2DBB21046D7
:105A6000AB420CD0194A0133802B14791E4C28BF4D
:105A70000023E45CE4B2D471127D072AF0D9DBB2D2
:105A80000370124B1A79140644BF7C22DA700F4B54
:105A90009A7C500706D5154A10780130C0B21070B4
:105AA00004229A74490610D5084B1A7952060CD56F
:105AB0000F4A002111700F4A126802B111709A79D1
:105AC00002F0DF029A713C22DA7030BD00A006407D
:105AD000808AFF1FFE88FF1F8089FF1FF888FF1F35
:105AE000888AFF1F828AFF1F0089FF1FF490FF1F13
:105AF000FC88FF1F848AFF1F1D4B1A6842F4006256
:105B00001A601C4A002313801B4A13801B4A13701F
:105B10001B4A13701B4A13701B4B40F213321A605E
:105B20004FF451725A60194BC0F344321A70C0F3EB
:105B300047125A7000F01F000422022198729A70D6
:105B4000D9745A7588221A743C22DA709A7842F015
:105B5000A0029A709A7902F0DF029A710C4B4022EF
:105B60001A70A3F22B334FF400421A60704700BF43
:105B700034800440948CFF1F928AFF1F9C8CFF1F6F
:105B8000968CFF1F908AFF1F0CB0044000B00640A7
:105B90002FE400E0134A937800F0030103F0EC03D4
:105BA0000B43410748BF43F01003937000F00F030D
:105BB000042B0C4903D18B7943F040038B7153794B
:105BC000C20603F0EF03074A48BF43F010035371C6
:105BD0009379810603F0EF0348BF43F010039371FC
:105BE000704700BF00B0064008B5114B1B681B058D
:105BF00000D408BD0F4B1A7802F0FF0312B101F078
:105C0000EFFCF7E70C4A4FF4004111600B4A0C49D6
:105C1000D37040F203120A604A600A4A13800A4AAB
:105C200013800A4B1B680BB101221A7008BD00BF1C
:105C300034800440908AFF1F84E100E000B00640F9
:105C40000CB00440948CFF1F928AFF1F8C8AFF1FA8
:105C500038B50446094B1B7803F0FF05002BF9D13A
:105C600020460121FFF7DCFA20462946FFF7B8FA63
:105C7000034B53F83420034B1A6038BD908AFF1F42
:105C800038A90000988CFF1F0D4A38B5146814F429
:105C900000624FF0000410D021280A4D0AD80A4AA9
:105CA000012152F830302B60FFF7BAFA2B681C70D4
:105CB000012038BD2C60204638BD104638BD00BFDD
:105CC000348004408C8AFF1F38A900000B4B1B68EE
:105CD00013F4006310D01728094B09D1094A40F288
:105CE000023111605A7B42F001025A730120704761
:105CF0005A7B02F0FE025A73002070473480044041
:105D000000B0064008B00440F8B51F4B1B681A05E8
:105D1000064638D51D4B9A7942F020029A711C4BE9
:105D20001B680BB101221A701A4B1C780134802CAD
:105D30001F4628BF0024184D2B78A34218D1FFF727
:105D4000A9F940280FDC114A13791B06F3D52B78EB
:105D500012490133802B28BF0023C95CDBB2C9B2D2
:105D6000D1712B70E7E7FF28E5DD01F039FCE2E7B0
:105D70000A4BF6B21E550A4B01221A70034BE4B2CD
:105D8000BC223C70DA70F8BD3480044000B006409C
:105D9000988CFF1F9C8CFF1F968CFF1F948AFF1FFF
:105DA000908AFF1F294B1B681A052DE9F04707460B
:105DB0008A4649D5264B9A7942F020029A71254BA2
:105DC0001B680BB101221A703D4607EB0A039D4286
:105DD00037D2DFF89080204E98F8004096F8009077
:105DE0000134802C28BF00245FFA89F9A1451DD118
:105DF000174BBC22DA70FFF74DF940280FDC144A2C
:105E000013791B060FD5337814490133802B28BF33
:105E10000023C95CDBB2C9B2D171337003E0FF2843
:105E200001DD01F0DDFB33784B45E4D00B4B15F879
:105E3000012B1A550A4B0122E4B21A7088F800406F
:105E4000C3E7034BBC22DA70BDE8F087348004401E
:105E500000B00640988CFF1F968CFF1F948AFF1F8E
:105E6000908AFF1F9C8CFF1F08B5034B1B7813B152
:105E700001F0B6FBF9E708BD908AFF1F064A074B01
:105E80001B781078DBB2C0B283422CBF7F3000F1A8
:105E9000FF30C01A704700BF968CFF1F9C8CFF1FFD
:105EA000054B1888054B1B8880B29BB2984238BFBF
:105EB00000F5C070C01A7047948CFF1F928AFF1FB4
:105EC000114B12491A880B8892B29BB29A4210B5B4
:105ED00016D00133B3F5C07F28BF00230C489CB215
:105EE000C05C0C800B490968C0B259B19A4238BFF6
:105EF00002F5C072D31A1A2B04DC00230B7010BDFC
:105F00004FF0FF3010BD00BF948CFF1F928AFF1F1F
:105F1000148BFF1F8C8AFF1F094B1A88094B1B88A3
:105F200092B29BB29A4208D00133B3F5C07F28BF2A
:105F30000023054AD05CC0B270474FF0FF30704775
:105F4000948CFF1F928AFF1F148BFF1F0C4B1B6842
:105F50001B0514D50B4BDA7802F0CB02DA70402225
:105F60005A74DA7842F03402DA70074B1A88074B19
:105F700092B21A80064B1B680BB100221A70704750
:105F80003480044000B00640928AFF1F948CFF1FAB
:105F90008C8AFF1F30B53E4B1A7912F0300F32D089
:105FA00072B69A7D02F0FF0022B9DA7940225A7463
:105FB00062B628E062B6374A3749138809889BB22F
:105FC00089B21446324AD5795A1CB2F5C07F28BF2F
:105FD00000228A42EDB202D0304B9D541346421E3D
:105FE00012F0FF00EED19AB222802D4A126852B10F
:105FF0008B4236BFC1F5C071C1EB03035B18272B81
:10600000C4BF01231370224BD978C9B20A0620D528
:106010001B791D061DD5234B234A1D781378EDB23D
:10602000DBB21046AB420CD0194A0133802B1479F5
:106030001E4C28BF0023E45CE4B2D471127D072A11
:10604000F0D9DBB20370124B1A79140644BF7C22DC
:10605000DA700F4B9A7C500706D5154A107801303C
:10606000C0B2107004229A74490610D5084B1A79F0
:1060700052060CD50F4A002111700F4A126802B166
:1060800011709A7902F0DF029A713C22DA7030BD09
:1060900000B00640948CFF1F928AFF1F148BFF1FD5
:1060A0008C8AFF1F9C8CFF1F968CFF1F948AFF1FFA
:1060B000C388FF1F908AFF1F988CFF1F174B1A6819
:1060C00042F480521A60164A00231380154A138046
:1060D000154A1380154A1380154A1370154A40F269
:1060E000133111604FF451715160134AC0F34431C0
:1060F0001170C0F3471100F01F005170907293703F
:1061000013742C23D3700D4B40226FF44B711A7013
:106110000B444FF400321A60704700BF34800440D3
:10612000A88FFF1FA68CFF1FB08FFF1FAA8FFF1F16
:10613000A48CFF1F08C0044000C0064031E400E00A
:10614000134A937800F0030103F0EC030B4341077B
:1061500048BF43F01003937000F00F03042B0C4969
:1061600003D18B7943F040038B715379C20603F05E
:10617000EF03074A48BF43F0100353719379810638
:1061800003F0EF0348BF43F010039371704700BF63
:1061900000C0064008B5114B1B68DB0400D408BDE5
:1061A0000F4B1A7802F0FF0312B101F019FAF7E76A
:1061B0000C4A4FF4003111600B4A0C49D37040F285
:1061C00003120A604A600A4A13800A4A13800A4B83
:1061D0001B680BB101221A7008BD00BF3480044057
:1061E000A48CFF1F84E100E000C0064008C004400A
:1061F000A88FFF1FA68CFF1FA08CFF1F38B5044679
:10620000094B1B7803F0FF05002BF9D12046012133
:10621000FFF706F820462946FEF7E2FF034B53F846
:106220003420034B1A6038BDA48CFF1F38A900002E
:10623000AC8FFF1F0D4A38B5146814F480524FF02C
:10624000000410D021280A4D0AD80A4A012152F828
:1062500030302B60FEF7E4FF2B681C70012038BD46
:106260002C60204638BD104638BD00BF3480044045
:10627000A08CFF1F38A900000B4B1B6813F4805340
:1062800010D00E28094B09D1094A40F202311160A1
:106290005A7B42F001025A73012070475A7B02F088
:1062A000FE025A73002070473480044000C006404C
:1062B00004C00440F8B51F4B1B68DA04064638D505
:1062C0001D4B1B680BB101221A701C4B1C88A4B219
:1062D0000134B4F5C07F1F4628BF0024184D2B8819
:1062E0009BB2A3421AD1FEF7D5FE402811DC154A15
:1062F00013791B06F2D52B8813499BB20133B3F5F2
:10630000C07F28BF0023C95C9BB2C9B2D1712B806A
:10631000E4E7FF28E2DD01F063F9DFE70A4BF6B2BC
:106320001E550A4B01221A70064BA4B2AC223C80C7
:10633000DA70F8BD34800440AC8FFF1FB08FFF1FB0
:10634000AA8FFF1F00C00640A88CFF1FA48CFF1F50
:1063500038B504464518AC4204D014F8010BFFF7D9
:10636000A9FFF8E738BDFFFF08B5034B1B7813B151
:1063700001F036F9F9E708BDA48CFF1F064A074B68
:106380001B8810889BB280B283422CBF00F27F1022
:1063900000F1FF30C01A7047AA8FFF1FB08FFF1F98
:1063A000054B1888054B1B8880B29BB2984238BFBA
:1063B00000F5C070C01A7047A88FFF1FA68CFF1F82
:1063C000114B12491A880B8892B29BB29A4210B5AF
:1063D00016D00133B3F5C07F28BF00230C489CB210
:1063E000C05C0C800B490968C0B259B19A4238BFF1
:1063F00002F5C072D31A1A2B04DC00230B7010BDF7
:106400004FF0FF3010BD00BFA88FFF1FA68CFF1FED
:10641000288EFF1FA08CFF1F094B1A88094B1B8871
:1064200092B29BB29A4208D00133B3F5C07F28BF25
:106430000023054AD05CC0B270474FF0FF30704770
:10644000A88FFF1FA68CFF1F288EFF1F054B1A88E1
:10645000054B92B21A80054B1B680BB100221A70D3
:10646000704700BFA68CFF1FA88FFF1FA08CFF1FC7
:1064700010B5314B1A79920623D5304AD879138852
:106480002F499BB201330988B3F5C07F28BF002391
:1064900089B28B42C0B203D02A49C85499B2118044
:1064A000294A116869B1294A128892B2934236BFCB
:1064B000C2F5C072C2EB03039B18272BC4BF012394
:1064C0000B701D4AD178C9B20C0618D5137918067D
:1064D00015D51F4B1D481C880388A4B29BB29C4253
:1064E00002D16C23D3700AE00133B3F5C07F28BF1B
:1064F0000023184CE45C9BB2E4B2D47103800E4BD1
:106500009A7C520706D5144A10780130C0B2107038
:1065100004229A744B060ED5074B1A7912F0400FDD
:10652000194608D00D4B00221A700D4B1B6803B1A1
:106530001A702C23CB7010BD00C00640A88FFF1F1F
:10654000A68CFF1F288EFF1FA08CFF1FAA8FFF1F86
:10655000B08FFF1FA88CFF1FF590FF1FA48CFF1F9B
:10656000AC8FFF1F21282BD8164B1B5CFF2B27D08D
:10657000154A02EBC000002142681160134A1068FE
:1065800040F020001060124A01201160114998402B
:106590000860114841F8040C104911604FF4A071D3
:1065A00001397FF4FDAF11688905FCD42022013A3E
:1065B0007FF4FDAF0A4A1BB232F8130080B2704775
:1065C0000020704748AA000038A900003880044025
:1065D00000500440085004400000020380014A00BB
:1065E00000510440F0B50C4B0C4C1A7842F00205F7
:1065F00004EBC50682F00102706009481A70067843
:10660000002E0CBF8827C82786F0010647EA014103
:10661000067044F83510F0BD1C90FF1F0080FF1F6E
:106620009490FF1F431E032B10B510D872B6094A71
:1066300052F8230048B1416842F82310064A018805
:1066400032F81340611A22F8131062B610BD002010
:1066500010BD00BF0C90FF1FF690FF1F01380328EC
:106660000AD872B6054B53F82030002013B1013020
:106670005B68FBE762B67047002070476090FF1FC1
:1066800010B572B60123174A1A4412F8012C1207EA
:106690001CD59900144A52F831402CB902EB43132F
:1066A00008305860114B09E041F0010152F83140C7
:1066B00064B902EBC103083058600D4B42F8313029
:1066C0000C4B1A78013A1A7062B610BD0133052BD3
:1066D000D9D162B6074B00221A70BDE8104000F015
:1066E000A7BB00BFA0AB00000080FF1F88004000D8
:1066F000C80040008A90FF1F431E032B30B532D8DC
:10670000194A400140F01000104472B6174CE25C88
:10671000032A09D8DFE802F0160218050830022221
:1067200013E00830042210E01148124A50F82340C8
:1067300014B940F8231002E052F82300416042F8F7
:1067400023100FE0032200E00522E25410F0080FAE
:1067500001F108030A8843600CBF8823C82343EA79
:106760000243036062B630BD0080FF1FC88FFF1F69
:106770006090FF1F7090FF1F2DE9F84FAB4F3C78E2
:10678000E4B214F0040F3D4619D0A94B1B78A3B115
:10679000A84A117801F0FF0321B1013BDBB213706D
:1067A00003B900BEA44A117801F0FF0329B1013BEF
:1067B000DBB213700BB900F04FFC04233B7004F004
:1067C000080303F0FF02002B00F067829B4B9C4CF8
:1067D0001A78D2B215094FEA920840F0E48104EB2E
:1067E000C803596854F83830C3F38303013B0C2BBA
:1067F00000F2D681DFE813F095019501D401D401B0
:10680000D401D401D401D401B001D401D401D40104
:106810000D008C4D0A684B688B486B6001218B4BD7
:1068200044F838302A60DFF85082017092B240F2AA
:10683000816000238242C8F800302361A36117D829
:10684000B2F5D06F80F01E81B2F5817F00F0CF806D
:1068500006D8802A00F0BA80822A00F0BB8031E19D
:1068600040F202339A4200F0D180B2F5A06F1CE0F2
:1068700042F22100824200F051810ED8B2F5086F39
:1068800000F09E80B2F5106F40F01C81684B6C4E9A
:10689000AA781A7006F180090AE042F221218A42A0
:1068A00000F0088142F221339A4200F00F8109E1A1
:1068B000336A1B0603D5706A083800F0B9FA083647
:1068C0004E45F5D10026B146DFF8B0A156F80A00D2
:1068D00028B1D0F804B000F0ABFA5846F8E74AF80F
:1068E00006005B4BDFF898A1F05056F80A0028B17B
:1068F000D0F804B000F09CFA5846F8E7554B4AF837
:106900000600F050544B23F81900544B19F803209B
:10691000023A032A08D8DFE802F002040204002247
:1069200000E0012203F8092009F10109B9F1040F7F
:1069300006F10406C8D14A4B00221A7001269A4675
:10694000484A494B3244334412F8012C9B0012F060
:10695000080F1A704FEA860925D000F04BFA38B1BB
:1069600004EB461308305860404B44F8393006E0D9
:106970009AF8003044F8390001338AF8003000F00A
:1069800039FA49F0010338B104EBC3020830506012
:106990002E4A44F8332006E044F833009AF80030D9
:1069A00001338AF8003049F00202013649F0030948
:1069B0000023052E44F8323044F83930C0D186E047
:1069C0001B4B2B4C1B7823700B4683E0284C237009
:1069D00063707EE0AA88042A74D8254C9200237044
:1069E0006370244B9B5C9E0773D5217071E0AA886D
:1069F00002F07F02042A65DC6B88002B62D19100D3
:106A00001C4A0A44117821F0020159E0AA8802F0D8
:106A10007F02042A56DC6B88002B53D19100154A63
:106A20000A44117841F002014AE000BF802007408B
:106A30009390FF1F1D90FF1F9590FF1F9020074010
:106A40000080FF1F8090FF1F9490FF1FC800400030
:106A5000B88FFF1F7090FF1FF690FF1FC88FFF1F9A
:106A60008A90FF1FA0AB000030C8011088004000D2
:106A70008B90FF1FC0200740B48FFF1F0C90FF1F9B
:106A80006090FF1F6A88A9889F4B53F8084CA3F1B8
:106A90000C00BCB133F80C6C964209D133F80A6C87
:106AA0008E4205D1120A032A0CBF2378038911E014
:106AB0000C33EAE7954A1168954A1160A978954A1E
:106AC000117004E0944B0F221A7027E000231C463B
:106AD00000E00223EE88B34238BF1E46402E34BF8A
:106AE0003546402520462946FFF77CFD761B2C4481
:106AF00003D1402D12D1354603E0402E34BF354638
:106B0000402520462946FFF76DFD761B2C4401D118
:106B1000402D03D1814AC8F8004016800122804BE5
:106B20003DE0804B1A8842F221039A4210D10023A3
:106B30007D4AC85C98540133072BF9D11368862B22
:106B400002D17A4B0F221A7000200146FFF74AFD4E
:106B5000774B44F8383023E0764E3568B5B1DFF82E
:106B6000BC81B8F80090B9F1400F34BF4C464024C6
:106B700028462146FFF736FDC4EB09039BB2A8F86F
:106B800000300BB9402C00D12B193360654B1A88AB
:106B9000B2F5A06F04D100225A709A78664B1A7031
:106BA00001225F4B6CE004EBC806013D736802F004
:106BB0000802A3F10800EDB202F0FF01002A36D06E
:106BC00000F036F95D485E4B50F82520EAB1516877
:106BD00040F8251002F108017160595D03290BD8B6
:106BE000DFE801F002040608032104E0022102E0CC
:106BF000052100E00421595516F0080F12880CBF3A
:106C00008823C82343EA024342E05A5D032A07D897
:106C1000DFE802F040400204002206E0012204E026
:106C200016F0080F0CBF022203225A5532E054F826
:106C30003820120C23F8082C22B3DFF834E123F8B3
:106C4000061C43F8041C5EF825303E4913B94EF883
:106C5000250002E051F8253058603B4B41F82500F3
:106C600033F815100A4423F8152000F0C3F810B1CA
:106C70000830706006E0354B44F838001A7801326D
:106C80001A7007E02A4B324A16F0080F08BF134665
:106C900044F8383008233B7070E5E0071FD52049E1
:106CA0002B482C4C02230B702B4B1A702B4B18606B
:106CB00098602B48D8601A619A615C60164B0D2071
:106CC00018702848FF2303702B700274264A137033
:106CD000264B9F221A7001230B70BDE8F88F210606
:106CE00004D50D4B0D221A7080232B70A20705D5F9
:106CF0001C4B1A78D2B21A7002232B70E30644BFE1
:106D000010232B70BDE8F88FB0AB0000F488FF1F94
:106D10000891FF1FA490FF1FC02007408890FF1F0D
:106D2000942007408090FF1F0091FF1F1D90FF1FC0
:106D3000C8004000B48FFF1F982007406090FF1FDD
:106D4000C88FFF1FB88FFF1FF690FF1F8A90FF1F8D
:106D500088004000CC8FFF1F1C90FF1F0080FF1F8A
:106D60002090FF1F882007408C2007408420074088
:106D70000C90FF1F08B500F071FC00221A4B002197
:106D8000D15098180832882A4160F7D1174A106804
:106D900040F48020106002F528326832C3F30720E7
:106DA0001070C3F307401B0E10751376FF2302F813
:106DB0001C3C02F8143C02F88C3C012302F8083C0D
:106DC00082F8641002F8183C094B70226FF450717D
:106DD0001A700B444FF400721A6003F1C04303F5BC
:106DE000C82310221A7008BD0080FF1F34800440A1
:106DF00049E400E072B60C4A1168B1FA81F30B2B3A
:106E000002D962B6002070474FF00040D84021EA16
:106E10000001116062B6054948225343C818002298
:106E2000CA504260704700BF7087FF1F0084FF1F79
:106E30000C4B4822C31AB3FBF2F30B2B11D80A4AAE
:106E4000127822B1094A12780AB1FFF719BC72B65A
:106E5000074A4FF0004121FA03F31168194311600A
:106E600062B670470084FF1F8A90FF1F9390FF1F38
:106E70007087FF1F10B5104C23686BB120684288E3
:106E8000531C0244147A0288934212D3FFF7D0FFB6
:106E9000094B00221A600DE0084B1B7813B94FF024
:106EA000FF3010BD0320FFF7BDFB20600028E5D1B7
:106EB000F5E74380204610BDA090FF1F9390FF1F71
:106EC00010B50B4C236813B123686BB902E0094B72
:106ED0001B7813B94FF0FF3010BD0320FFF7A2FB62
:106EE00020600028F0D1F5E75A881344187A10BDC5
:106EF000A090FF1F9390FF1F044B9888044B1B68C2
:106F00001BB11A885B88D31A18447047F690FF1F8C
:106F1000A090FF1F2DE9F8432D4E012307460C4694
:106F20003370002C4FD02B4D2B68A9462BBB4AF257
:106F3000F928294B1B7803F0FF020BB9327015E0DA
:106F40000420FFF78BFB072808D801233370FFF7D5
:106F500051FFC9F8000080B91D4B1870B8F1010845
:106F60001E4B01D01A782AB101221A704FF0FF305F
:106F7000BDE8F88300F034FBDBE72968174A48884E
:106F800000231370C0F14002944238BF224600F142
:106F9000080C10448C444880A41A934204D0F85C36
:106FA0000CF803000133F8E71F444B883F2B06D948
:106FB00040230B800420FFF79FFB00232B60084B2E
:106FC00005221A70ADE734702046BDE8F88300BF93
:106FD0009690FF1F9890FF1F9390FF1F9C90FF1F9C
:106FE0009590FF1F07B502AB012103F8010D18466C
:106FF000FFF790FF03B05DF804FBFFFF2DE9F041C0
:10700000114B1B78F3B1114E114B3468114D012710
:107010001F7098464CB1002763882F70042023808E
:107020002146FFF769FB376009E0FFF7E3FE014601
:1070300020B104202C70FFF75FFB00E02F700023CD
:1070400088F80030BDE8F0819390FF1F9890FF1FF3
:107050009690FF1F9590FF1F38B50E4B1B7803F0DD
:10706000FF05ABB90C4C216831B14B880B80042073
:10707000FFF742FB256038BDFFF7BCFE014620B19B
:107080000420BDE83840FFF737BB044B01221A70DB
:1070900038BD00BF9690FF1F9890FF1F9590FF1F6F
:1070A00008B50368C9B21B68984708BD08B50368EE
:1070B000C9B21B68984708BD08B50368C9B21B6808
:1070C000984708BD08B50368C9B21B68984708BD52
:1070D0004B0803F1376000F5D830B0FBF1F0FEF754
:1070E00021BA10B54B0803F1376000F5D8301446CB
:1070F000B0FBF1F0FEF716FA2046BDE81040FEF7AF
:107100005FBAFEF787BA0846FEF7B8BA08B5084670
:10711000FEF7D0FA003018BF012008BD08B50846B8
:10712000FEF7EAFA003018BF012008BDFEF7D6BB13
:10713000FEF710BCFEF7E2BBFEF7B4BBFEF724BCC3
:10714000FEF7BABB08B50846FEF7FCFA012008BDF9
:1071500008B50846FEF7F6FA012008BD10B5084646
:1071600014461146FEF73CFB204610BD38B50846D4
:107170000D4600F01EFF044621462846FEF730FB70
:10718000204638BD7047FFFF044B00221A714FF4B0
:107190007A711A73024A99601A607047A890FF1FAB
:1071A00078AA000008B50368C9B21B68984708BDF3
:1071B00008B50368C9B21B68984708BD08B50368DD
:1071C000C9B21B68984708BD08B50368C9B21B68F7
:1071D000984708BD4B0803F1376000F5D830B0FB85
:1071E000F1F0FEF789BC10B54B0803F1376000F5EC
:1071F000D8301446B0FBF1F0FEF77EFC2046BDE827
:107200001040FEF7C7BCFEF7EFBC0846FEF720BDF6
:1072100008B50846FEF738FD003018BF012008BD4C
:1072200008B50846FEF752FD003018BF012008BD22
:10723000FEF736BEFEF770BEFEF742BEFEF714BE86
:10724000FEF784BEFEF71ABE08B50846FEF75CFDE1
:10725000012008BD08B50846FEF756FD012008BD0F
:1072600010B5084614461146FEF79CFD204610BD99
:1072700038B508460D4600F09CFE044621462846D7
:10728000FEF790FD204638BD7047FFFF044B0022FB
:107290001A714FF47A711A73024A99601A60704732
:1072A000B890FF1FD0AA000008B50368C9B21B68D8
:1072B000984708BD08B50368C9B21B68984708BD60
:1072C00008B50368C9B21B68984708BD08B50368CC
:1072D000C9B21B68984708BD4B0803F1B76000F5B9
:1072E0005840B0FBF1F0FEF7E9BE10B54B0803F1D2
:1072F000B76000F558401446B0FBF1F0FEF7DEFE33
:107300002046BDE81040FEF71BBFFEF743BF08460E
:10731000FEF774BF08B50846FEF78CFF003018BFB3
:10732000012008BD08B50846FEF7A6FF003018BFCB
:10733000012008BDFFF734B8FFF76EB8FFF740B87B
:10734000FFF712B8FFF782B8FFF718B808B508467C
:10735000FEF7B0FF012008BD08B50846FEF7AAFFFA
:10736000012008BD10B5084614461146FEF7F0FF8F
:10737000204610BD38B508460D4600F01AFE0446FA
:1073800021462846FEF7E4FF204638BD7047FFFF40
:10739000044B00221A714FF47A711A73024A9960F1
:1073A0001A607047C890FF1F28AB000008B5F9F7B6
:1073B00059F8F9F7C3F900F013F9FAE700F0D8BC6F
:1073C00000F0DEBC2DE9F04100258C688AB007464C
:1073D00088462E4694B12B46404601A9212200F052
:1073E000E6F83B68202C34BF224620225B683846F2
:1073F00001A91544A41A98470644EBE730460AB0A1
:10740000BDE8F08107B5064B1B88ADF80430036872
:1074100001A95B680222984703B05DF804FB00BF36
:1074200078AB000008B503685B689847002008BD8A
:107430000EB403B503AA52F8041B019200F0AAFE91
:1074400002B05DF804EB03B0704770B505468AB032
:1074500022B90368C9B21B6898472CE0012A08BF0B
:107460000A2221B930228DF82520212413E021247D
:10747000B1FBF2F002FB1011C9B209290AAE94BFA8
:10748000303137312644C9B206F8241C014610B108
:10749000013CE4B2ECE733B1013CE4B20AAB234473
:1074A0002D2203F8242C2B6801A95B68284621446F
:1074B000C4F1220298470AB070BD0029BABF494200
:1074C0002D2300230A22FFF7C0BFFFF715BDFFF7EA
:1074D000D1BCFFF7F5BCFFF791BD0846FFF782BDB1
:1074E00008461146FFF716BD7047FFFF044B002208
:1074F0001A714FF47A711A73024A99601A607047D0
:10750000D890FF1F88AB000010B50446006800F05B
:1075100037FC204610BD38B504460D4600680131E1
:1075200000F00EFD10B184E82100012038BD436851
:107530008B4210B5044606D2FFF7EDFF20B1A368D9
:107540000BB922681370012010BDF8B504460F4630
:10755000154622B9036803B11A7000230BE01146E7
:10756000FFF7E5FF064640B9206810B100F008FCBF
:10757000266000236360A36004E0A56020683946AC
:1075800000F00FFD2046F8BD38B500230446036027
:107590004360836003730D4639B1084600F009FD6E
:1075A000294602462046FFF7D0FF204638BD38B5B1
:1075B0000C469AB191B181688B4202D300232370AB
:1075C00038BDC91A551E8D4228BF0D4601682A468E
:1075D0001944204600F00CFD0023635538BDFFFF21
:1075E00010B50E4C2378BBB901232370FFF784FC40
:1075F00008B1FFF779FFFEF771F908B1FFF7C2FD97
:10760000FEF74EFC08B1FFF73FFEFEF7C9FE08B1DA
:10761000FFF7BCFE0023237010BD00BFE890FF1FE2
:1076200010B50023B0FBF2F402FB1400092894BF4C
:1076300030303730C0B2C85420460CB10133F1E7C6
:10764000CA18547022469A4206DA885CCC5C8C5484
:10765000C8540132013BF6E7084610BD1FB572B6AB
:10766000154B70221A70154A412111700F2102F832
:10767000011C80221A701A781206FCD5104B18686B
:1076800062B6104B984298BF0A2301AC98BF58438A
:1076900021460A22FFF7C4FF0023E15C0A4A29B110
:1076A00002EB430001330A2B4180F6D101335B002A
:1076B000137004B010BD00BF00000240070002407C
:1076C000080002407F969800FC87FF1F80F0004072
:1076D00002E000BF81F0004142001FBF5FEA4103AA
:1076E00092EA030F7FEA226C7FEA236C6AD04FEAAA
:1076F0001262D2EB1363C1BFD218414048404140EF
:10770000B8BF5B42192B88BF704710F0004F40F4A0
:10771000000020F07F4018BF404211F0004F41F4BC
:10772000000121F07F4118BF494292EA030F3FD088
:10773000A2F1010241FA03FC10EB0C00C3F120039B
:1077400001FA03F100F0004302D5494260EB40002A
:10775000B0F5000F13D3B0F1807F06D340084FEA95
:10776000310102F10102FE2A51D2B1F1004F40EB8A
:10777000C25008BF20F0010040EA030070474900F2
:1077800040EB000010F4000FA2F10102EDD1B0FABD
:1077900080FCACF1080CB2EB0C0200FA0CF0AABFB2
:1077A00000EBC25052421843BCBFD0401843704750
:1077B00092F0000F81F4000106BF80F40000013256
:1077C000013BB5E74FEA41037FEA226C18BF7FEA2D
:1077D000236C21D092EA030F04D092F0000F08BF6F
:1077E0000846704790EA010F1CBF0020704712F056
:1077F0007F4F04D1400028BF40F00040704712F195
:1078000000723CBF00F50000704700F0004343F0F9
:10781000FE4040F4000070477FEA226216BF08462F
:107820007FEA23630146420206BF5FEA412390EAF2
:10783000010F40F4800070474FF0000304E000BFE8
:1078400010F0004348BF40425FEA000C08BF704799
:1078500043F0964301464FF000001CE050EA01025D
:1078600008BF70474FF000030AE000BF50EA010272
:1078700008BF704711F0004302D5404261EB41015F
:107880005FEA010C02BF84460146002043F0B64384
:1078900008BFA3F18053A3F50003BCFA8CF2083AA9
:1078A000A3EBC25310DB01FA02FC634400FA02FCB2
:1078B000C2F12002BCF1004F20FA02F243EB0200B9
:1078C00008BF20F00100704702F1200201FA02FC1B
:1078D000C2F1200250EA4C0021FA02F243EB02000E
:1078E00008BF20EADC7070474FF0FF0C1CEAD05252
:1078F0001EBF1CEAD15392EA0C0F93EA0C0F6FD013
:107900001A4480EA010C400218BF5FEA41211ED0F0
:107910004FF0006343EA501043EA5111A0FB0131DC
:107920000CF00040B1F5000F3EBF490041EAD371B1
:107930005B0040EA010062F17F02FD2A1DD8B3F12D
:10794000004F40EBC25008BF20F00100704790F09C
:10795000000F0CF0004C08BF49024CEA502040EAEE
:1079600051207F3AC2BFD2F1FF0340EAC2507047B4
:1079700040F400004FF00003013A5DDC12F1190FF2
:10798000DCBF00F000407047C2F10002410021FA64
:1079900002F1C2F1200200FA02FC5FEA310040F17C
:1079A000000053EA4C0308BF20EADC70704792F0F5
:1079B000000F00F0004C02BF400010F4000F013A2D
:1079C000F9D040EA0C0093F0000F01F0004C02BF28
:1079D000490011F4000F013BF9D041EA0C018FE797
:1079E0000CEAD15392EA0C0F18BF93EA0C0F0AD09D
:1079F00030F0004C18BF31F0004CD8D180EA0100C3
:107A000000F00040704790F0000F17BF90F0004F5B
:107A1000084691F0000F91F0004F14D092EA0C0F3D
:107A200001D142020FD193EA0C0F03D14B0218BFD0
:107A3000084608D180EA010000F0004040F0FE4016
:107A400040F40000704740F0FE4040F440007047B2
:107A50004FF0FF0C1CEAD0521EBF1CEAD15392EA31
:107A60000C0F93EA0C0F69D0A2EB030280EA010C21
:107A700049024FEA402037D04FF0805343EA1111BA
:107A800043EA10130CF000408B4238BF5B0042F118
:107A90007D024FF4000C8B4224BF5B1A40EA0C00BD
:107AA000B3EB510F24BFA3EB510340EA5C00B3EBEF
:107AB000910F24BFA3EB910340EA9C00B3EBD10FDD
:107AC00024BFA3EBD10340EADC001B0118BF5FEA2F
:107AD0001C1CE0D1FD2A3FF650AF8B4240EBC25058
:107AE00008BF20F0010070470CF0004C4CEA502019
:107AF0007F32C2BFD2F1FF0340EAC250704740F468
:107B000000004FF00003013A37E792F0000F00F059
:107B1000004C02BF400010F4000F013AF9D040EAD7
:107B20000C0093F0000F01F0004C02BF490011F46B
:107B3000000F013BF9D041EA0C0195E70CEAD15363
:107B400092EA0C0F08D142027FF47DAF93EA0C0F4A
:107B50007FF470AF084676E793EA0C0F04D14B022E
:107B60003FF44CAF08466EE730F0004C18BF31F0E0
:107B7000004CCAD130F000427FF45CAF31F00043DA
:107B80007FF43CAF5FE700BF4FF0FF3C06E000BF73
:107B90004FF0010C02E000BF4FF0010C4DF804CD96
:107BA0004FEA40024FEA41037FEA226C18BF7FEAA6
:107BB000236C11D001B052EA530C18BF90EA010FA8
:107BC00058BFB2EB030088BFC81738BF6FEAE17037
:107BD00018BF40F0010070477FEA226C02D15FEAD3
:107BE000402C05D17FEA236CE4D15FEA412CE1D03F
:107BF0005DF8040B704700BF844608466146FFE706
:107C00000FB5FFF7C9FF002848BF10F1000F0FBDE7
:107C10004DF808EDFFF7F4FF0CBF012000205DF8E0
:107C200008FB00BF4DF808EDFFF7EAFF34BF012065
:107C300000205DF808FB00BF4DF808EDFFF7E0FFFE
:107C400094BF012000205DF808FB00BF4DF808ED4F
:107C5000FFF7D2FF94BF012000205DF808FB00BFB2
:107C60004DF808EDFFF7C8FF34BF012000205DF894
:107C700008FB00BF4FEA4002B2F1FE4F0FD34FF0B6
:107C80009E03B3EB12620DD94FEA002343F0004389
:107C900010F0004F23FA02F018BF404270474FF037
:107CA0000000704712F1610F01D1420205D110F0BE
:107CB000004008BF6FF0004070474FF00000704771
:107CC00042000ED2B2F1FE4F0BD34FF09E03B3EB46
:107CD000126209D44FEA002343F0004323FA02F072
:107CE00070474FF00000704712F1610F01D142025E
:107CF00002D14FF0FF3070474FF00000704700BFD7
:107D000000210A2200F008BA00210A2200F004BA79
:107D10000A46034903460868194600F06BB800BFDD
:107D20007488FF1F70B50E4B0E4DED1AAD10002478
:107D30001E46AC4204D056F8242090470134F8E7A0
:107D400003F02AF8084D094BED1AAD1000241E4629
:107D5000AC4204D056F8242090470134F8E770BDB7
:107D6000A4AD0000A4AD0000B8AD0000A4AD0000BB
:107D7000024B0146186800F08FB800BF7488FF1FDF
:107D8000024B0146186800F043B800BF7488FF1F1B
:107D900010B5C9B202449042034606D01C788C420A
:107DA00000F10100F7D1184610BD002010BD81423E
:107DB00070B501D300230EE08C18A042FAD28518CA
:107DC000134613F1FF3305D3514266182944F65C7C
:107DD000CE54F6E770BD934203D0CC5CC45401335B
:107DE000F9E770BD02440346934202D003F8011B39
:107DF000FAE7704738B502FB01F4214600F04CF871
:107E0000054618B100212246FFF7ECFF284638BD91
:107E100030B500293CD051F8042C0B1F1D49002A15
:107E2000B8BF9B180A680C4612B95A600B6030BD87
:107E300093420DD219685818904203D15A581144F0
:107E4000426819605A60236030BD994203D80A46DF
:107E500051680029F9D1146815199D420AD11B688F
:107E60002344D0188842136012D108680344136079
:107E70004B680CE002D90C23036030BD18681C1855
:107E80008C4203D10C6849682044186059605360E3
:107E900030BD00BFF090FF1F70B5CD1C25F003056D
:107EA00008350C2D38BF0C25002D06463FDB8D42D2
:107EB0003DD3214B1C6818462146A1B10B685B1BC2
:107EC0000ED40B2B03D90B60CC18CD501FE08C4285
:107ED00002D1626802601AE04B6863600C4616E0EB
:107EE0000C464968E9E7154C23681BB9304600F099
:107EF00031F820602946304600F02CF8431C01463A
:107F000015D0C41C24F0030484420AD1256004F176
:107F10000B00231D20F00700C31A0BD05A42E25079
:107F200070BD3046611A00F015F80130EED10C2317
:107F30003360002070BD00BFF090FF1FEC90FF1F6A
:107F40000A46034903460868194600F001BA00BF13
:107F50007488FF1F38B5064C002305460846236089
:107F6000FDF786F8431C02D1236803B12B6038BDAE
:107F70000C91FF1FC9B2024610F8013B1BB18B42A6
:107F8000F9D1104670470029FBD01846704710F809
:107F9000012B11F8013B012A28BF9A42F7D0D01AD1
:107FA0007047034611F8012B03F8012B002AF9D181
:107FB0007047034613F8012B002AFBD1181A013829
:107FC000704770B592B10B4605461C7810F8016BEE
:107FD000B44201F1010101D1012A03D128781B78B3
:107FE000C01A70BD013A002CEDD1F7E7104670BD04
:107FF00010B5034632B111F8014B03F8014B013AB9
:10800000002CF7D11A44934203D0002103F8011B3E
:10801000F9E710BD84463F482DE9F04FD0F80080C5
:108020000E46344614F8015B08EB0500407800F07A
:10803000080000F0FF0708B12646F2E72D2D03D116
:10804000B41C7578012703E02B2D04BF7578B41C90
:1080500033F010000DD1302D08D1207800F0DF0072
:10806000582851D165781023023402E0002B08BF54
:108070000A23002F0CBF6FF0004A4FF0004ABAFBF2
:10808000F3F9002603FB19AA304608EB050B9BF811
:1080900001B01BF0040F01D0303D0BE01BF0030BCF
:1080A0001BD0BBF1010F14BF4FF0570B4FF0370B34
:1080B000CBEB05059D4210DAB6F1FF3F0AD04845EB
:1080C00006D801D1554503DC03FB0050012601E031
:1080D0004FF0FF3614F8015BD7E7731C0CD1002F6B
:1080E0004FF022030CBF6FF000404FF00040CCF87F
:1080F00000302AB9BDE8F08F07B1404242B106B165
:10810000611E1160BDE8F08F002B08BF0823B0E7A7
:10811000BDE8F08F7888FF1F30B51346044A054646
:108120000C46106829462246BDE83040FFF772BF72
:108130007488FF1F2DE9F041ADF5047D1D464FF415
:1081400000730F4690460393044618B183690BB938
:1081500000F094F804AE00952046314603AA434649
:1081600000F05FF9054670B1204639462A46039B68
:1081700000F01EF8B542039003D020462946FFF7D1
:1081800047FE039801E04FF0FF300DF5047DBDE898
:10819000F081FFFF30B51346044A05460C461068CF
:1081A00029462246BDE83040FFF7C4BF7488FF1F50
:1081B00038B5074C054600202060084611461A468F
:1081C000FFF730F9431C02D1236803B12B6038BD9F
:1081D0000C91FF1FF8B5074600F1480494B1A5685B
:1081E0006668013E0CD4AB89012B07D9B5F90E3076
:1081F000013303D03846294600F0D6F96835F0E758
:108200002468EBE7F8BDFFFF002310B504460360C8
:108210004360836081814366C281036143618361FE
:1082200019465C300822FFF7DDFD054B6362054B04
:10823000A362054BE362054B2462236310BD00BFBC
:108240009D830000BF830000F78300001B840000B3
:1082500070B54B1E68255D430E4605F17401FFF7AE
:108260001BFE044640B1002180E842000C30A060B3
:1082700005F16802FFF7B6FD204670BD836910B5B1
:10828000044633BB8364C3640365124B124A1B6804
:108290008262984204BF0123836100F01FF860608E
:1082A000204600F01BF8A060204600F017F80421DB
:1082B000E06000226068FFF7A7FFA06809210122A3
:1082C000FFF7A2FFE06812210222FFF79DFF0123C2
:1082D000A36110BDFCAB0000D5810000F8B51B4BBD
:1082E0001E68B369074613B93046FFF7C7FF483623
:1082F000B4687368013B04D4B4F90C5075B16834A8
:10830000F8E733682BB938460421FFF7A1FF306046
:1083100008B13668ECE70C233B60F8BD4FF6FF73FD
:10832000E3810123A38165662560A5606560256101
:108330006561A56104F15C0029460822FFF752FD42
:108340006563A563A564E5642046F8BDFCAB000049
:10835000F8B5064614460D4621B91146BDE8F84069
:10836000FFF79ABD1AB9FFF753FD2046F8BD00F09C
:1083700057F9A0420ED230462146FFF78DFD074641
:1083800050B129462246FCF7BBFA30462946FFF792
:108390003FFD01E02846F8BD3846F8BD10B50C4653
:1083A000B1F90E1000F046F9002803DB636D0344B9
:1083B000636510BDA38923F48053A38110BD2DE90B
:1083C000F0411D468B89DB0507460C46164605D550
:1083D000B1F90E100022022300F010F9A389B4F9BC
:1083E0000E1023F48053A381384632462B46BDE855
:1083F000F041FFF7DDBE10B50C46B1F90E1000F0EC
:10840000FDF8431CA38903D123F48053A38110BD3D
:1084100043F48053A381606510BDB1F90E1000F0E4
:108420002FB830B515469BB0146829B124B14FF46C
:10843000C162ADF80C2005E04FF422720024ADF8C3
:108440000C202146002C0091049103DA8B23036059
:10845000002012E04FF6FF72ADF80E2069461A4672
:108460001E9B0294059400F053F9031E4FF0000088
:1084700003DB2B60009B187004981BB030BDFFFF1E
:1084800038B5064C0023054608462360FCF7FAFD84
:10849000431C02D1236803B12B6038BD0C91FF1F30
:1084A0008A892DE9F041054610070C4657D44B68E0
:1084B000002B02DC0B6C002B18DDE66AB6B102F46F
:1084C0008052002392B22F682B600AB1626D10E0D7
:1084D000216A28460123B047411C024609D12B6876
:1084E0003BB11D2B01D0162B46D12F600020BDE8DB
:1084F000F081A3895B0705D56368D21A636B0BB162
:10850000236CD21AE66A216A28460023B047461C2B
:10851000A28905D12B681BB11D2B01D0162B19D1B7
:1085200000236360D1042369236004D5421C01D178
:108530002B6803B96065616B2F600029D6D004F108
:108540004403994202D02846FFF762FC0020606392
:10855000BDE8F08142F04002A281BDE8F0810E69E1
:10856000002EC3D00B680E60C6EB030893070CBF48
:108570004B6900238B6012E0A38943F04003A38181
:108580004FF0FF30BDE8F081A76A216A28463246E5
:108590004346B8470028EFDD0644C0EB0808B8F1B1
:1085A000000FF1DCA2E7FFFF38B50B6905460C466A
:1085B000DBB118B183690BB9FFF760FE0C4B9C422D
:1085C00001D16C6808E00B4B9C4201D1AC6803E020
:1085D000094B9C4208BFEC68B4F90C302BB128461B
:1085E0002146BDE83840FFF75BBF002038BD00BF23
:1085F00004AD000024AD000044AD000038B5074CC8
:10860000054600202060084611461A46FCF73DFD4D
:10861000431C02D1236803B12B6038BD0C91FF1FAE
:1086200051F8040C002802DA04390B5818440438B5
:108630007047FFFF38B5074C05460020206008460C
:1086400011461A46FCF71CFD431C02D1236803B1F6
:108650002B6038BD0C91FF1F2DE9F0478D68AB42B0
:1086600081460C4692461F4643D38B8913F4906F84
:108670003DD026680969C1EB06086669022206EB4F
:10868000460696FBF2F608F101023A44964238BFDC
:1086900016465B050FD53146FFF7FEFB054698B140
:1086A00021694246FCF72CF9A38923F4906343F037
:1086B0008003A38113E03246FFF74AFE054670B9F6
:1086C00048462169FFF7A4FB0C23C9F80030A389B1
:1086D00043F04003A3814FF0FF30BDE8F0872561F0
:1086E00066614544C8EB06062560A6603D46AF427C
:1086F00000D23D462A4620685146FFF758FBA36842
:108700005B1BA36023681D4425600020BDE8F08743
:108710002DE9F0439DB0074603938B891C060D4657
:1087200016460CD50B6953B94021FFF7B5FB2860FD
:10873000286110B90C233B60C8E040236B61002323
:10874000099320238DF8293030238DF82A303346C1
:108750001C4613F8012B1AB9B4EB06090FD002E03E
:10876000252AF5D1F8E73846294632464B46FFF729
:1087700073FF013000F0A580099B4B4409932378D7
:10878000002B00F09E8000234FF0FF3204930793EC
:10879000059206938DF853301A9304F101094C4663
:1087A0004D4E217830460522FFF7F2FA09F1010912
:1087B000049B28B1861B0120B04003430493EEE7DD
:1087C000D90644BF20228DF853201A0744BF2B221C
:1087D0008DF8532022782A2A02D0079B21460EE0EA
:1087E000039A111D12680391002A01DB079204E02D
:1087F000524243F002030792049301340AE00C460C
:1088000001312278303A092A03D80A2000FB0323D9
:10881000F5E7079323782E2B1AD163782A2B0AD1F8
:10882000039B1A1D1B680392002B04F10204B8BFBE
:108830004FF0FF330BE0611C00230C46013122781E
:10884000303A092A03D80A2000FB0323F5E70593F1
:10885000224E217830460322FFF79AFA30B1861B68
:10886000049B4020B04003430493013421781C480A
:108870008DF828100622661CFFF78AFA88B1194B7A
:1088800033B9039B073323F007030833039314E042
:1088900003AB0093384604A92A46134BAFF300807C
:1088A00007E003AB0093384604A92A460E4B00F0BC
:1088B0008FF8B0F1FF3F804603D0099B43440993F2
:1088C00045E7AB895B0601D4099801E04FF0FF3022
:1088D0001DB0BDE8F08300BF64AD00006AAD0000CC
:1088E0006EAD000000000000598600002DE9F8433D
:1088F00015461F468A680B69DDF820809A42A8BF9A
:1089000013462B6091F8432006460C460AB101330A
:108910002B602368990602D52B6802332B602368ED
:1089200013F006091DD094F843302268003318BFB5
:10893000012392061FD5E1185A1C302081F843000C
:10894000224494F8451082F84310023313E0304675
:10895000394604F119020123C047013007D009F15B
:108960000109E2682B68D31A9945F0DBDBE74FF089
:10897000FF30BDE8F8833046394604F14302C04772
:108980000130F4D023682A68E16803F00603042B61
:1089900008BFC2EB01052369A2680CBF25EAE57593
:1089A00000259A42C4BFC3EB0203ED184FF0000943
:1089B000A9450ADA3046394604F11A020123C047B4
:1089C0000130D4D009F10109F2E70020BDE8F883B5
:1089D0002DE9FF470E7E0C9D6E2E80460C4691467B
:1089E0009A4601F1430000F0A58011D8632E22D0F1
:1089F00009D8002E00F0AF80582E40F0BF8081F8DB
:108A000045607B4A4FE0642E1ED0692E1CD0B5E035
:108A1000732E00F0A48009D86F2E2BD0702E40F05A
:108A2000AD800B6843F020030B6038E0752E21D039
:108A3000782E34D0A2E02B681A1D1B682A6001F141
:108A4000420781F842309DE022682B6812F0800FC7
:108A500003D01A1D2A601D6805E05106F9D51A1DBC
:108A60002A60B3F90050002D39DA2D236D4284F8C5
:108A7000433034E022682B6812F0800F03D01A1DB7
:108A80002A601D6804E05206F9D51A1D2A601D8867
:108A9000237E574A6F2B14BF0A2308231BE0782339
:108AA000544A84F845302368296813F0800F01F197
:108AB00004062E6001D00D6802E05F06FBD50D882C
:108AC000DE0744BF43F0200323601DB9236823F071
:108AD000200323601023002184F8431001E0444A5E
:108AE0000A236668A660002E03DB216821F00401DA
:108AF000216005B96EB104F14201B5FBF3F603FB49
:108B000016550F46555D01F801593546002EF4D132
:108B100000E00746082B0AD12368DD0707D5626805
:108B200023699A4203DC302307F8013C013FC01B54
:108B300020612CE009682B68626911F0800F04D075
:108B4000191D29601B681A6005E04906F8D5191D32
:108B500029601B681A8000232361074617E02B68F1
:108B60001A1D2A601F683846FFF723FA63682061E0
:108B7000984288BF23612369636005E004F14207DE
:108B800084F8426001232361002384F84330CDF848
:108B900000A04046214603AA4B46FFF7A7FE01303E
:108BA00002D14FF0FF301FE0404649463A46236964
:108BB000D0470130F5D023689B0705D4E068039BBC
:108BC0009842B8BF18460FE00025E268039BD31A0D
:108BD0009D42F3DA4046494604F119020123D04789
:108BE0000130DED00135F0E704B0BDE8F08700BF0A
:108BF00075AD000086AD00005B4254204E4F5420FE
:108C000050524553454E545D0041542B55415254EA
:108C10003D25642C302C30000D0A004F4B00415490
:108C20000041542B4E414D453F0041542B5053576A
:108C3000443F005B4D41494E4252445F554E5355AF
:108C400050525445445D0041542B4E414D453D2505
:108C5000730041542B505357443D25303469004331
:108C6000616C6C6F63206661696C20320044756DC5
:108C700070696E672043697263756C6172206275FA
:108C8000666665725F006275666665725F2073690D
:108C90007A652069733A2025640A00252E327820EF
:108CA00000FFFFFFFFFFFFFF0000000000000000CB
:108CB0009150000039130000511300000000000023
:108CC00018011EFF03FFFFFF00000000000000006E
:108CD0007913000045130000651300000000000038
:108CE0005B74696D656F75745D0A005B25645D205A
:108CF0005B25645D0A005B706172616D735F636F19
:108D0000756E742025645D205B25645D0A00556ED8
:108D10006B6E6F776E20737461746520696E20636B
:108D2000616C6C6261636B20696E20636C73436F6E
:108D30006E736F6C652121210A005363616E6E6949
:108D40006E6720696E2070726F677265732E205592
:108D5000736520636F6D6D616E6420277374617439
:108D600075732720746F206C6973742049447320D5
:108D7000666F756E642E00596573004E6F00536503
:108D8000656420526F626F746963732045524F535C
:108D9000204669726D776172650A00426F61726484
:108DA000206D6F64656C2025640A00426F617264F7
:108DB00020485720436F6E66696775726174696FEA
:108DC0006E2025640A004669726D776172652076AF
:108DD000657273696F6E2025640A0053657269615C
:108DE0006C204E756D62657220252E3278252E32EC
:108DF00078252E32780A0043757272656E7420737E
:108E0000656E736F72207265736973746F7220760A
:108E1000616C75653A2025640A00426F61726420B6
:108E2000697320636F6E6669677572656420746F1D
:108E3000206F7065726174652077697468203132C3
:108E4000626974207265736F6C7574696F6E2E0A37
:108E500000426F61726420697320636F6E66696798
:108E60007572656420746F206F706572617465201F
:108E700077697468203130626974207265736F6C31
:108E80007574696F6E2E0A000A45787465726E619A
:108E90006C2062757320636F6D6D756E69636174AC
:108EA000696F6E2073657474696E67733A200A0087
:108EB000426F6172642062757320646576696365D0
:108EC0002049443A2025640A0052657475726E2068
:108ED00064656C61792074696D653A202564205B56
:108EE0002564206D6963726F736563735D0A005357
:108EF00074617475732072657475726E206C65761A
:108F0000656C3A2025640A005573696E67205458D1
:108F100020456E61626C652070696E3A2025730A87
:108F2000000A496E7465726E616C2062757320630D
:108F30006F6D6D756E69636174696F6E20736574B2
:108F400074696E67733A20000A496E7465726E61C7
:108F50006C206275732042617564207261746520B3
:108F600073657474696E673A202564203D2025641A
:108F7000204250530A000A4120426C7565746F6F9D
:108F8000746820636F6D6D756E69636174696F6E6F
:108F9000206D6F64756C65206973207072657365F0
:108FA0006E743A0A00426C7565746F6F7468204382
:108FB0004F4D4D20426175642073657474696E670E
:108FC000202564203D202564204250530A00426C35
:108FD0007565746F6F746820646576696365206E6B
:108FE000616D653A202573200A00426C7565746FC7
:108FF0006F74682064657669636520636F64653AA1
:109000002025303464200A000A4E6F20426C7565BA
:10901000746F6F746820636F6D6D756E69636174D2
:10902000696F6E206D6F64756C652064657465632F
:109030007465642E0A004F6E004F666600426F61D1
:109040007264205374617475733A0A00496E7465D2
:10905000726E616C2054656D7065726174757265B5
:109060003A09256420646567430A0045787465728F
:109070006E616C20537570706C7920566F6C7461E2
:1090800067653A0925642E2564560A00436F6E66AB
:1090900069677572656420566F6C746167652069D5
:1090A0006E20496E7465726E616C204275733A0968
:1090B0002564560A0A00506F736974696F6E2053F5
:1090C000656E736F722057416464756374696F6E67
:1090D0003A0925640A00506F736974696F6E2053F2
:1090E000656E736F722057466C6578696F6E3A09CA
:1090F00025640A0050616C6D204F70746963616C67
:109100002053656E736F7220696E7374616C6C6549
:10911000643A0925730A0050616C6D204F707469C0
:1091200063616C2053656E736F7220416D62696577
:109130006E74204C696768743A0925640A005061AE
:109140006C6D204F70746963616C2053656E736F32
:109150007220436F6D707574656420526561646937
:109160006E673A0925640A00436170616369746936
:1091700076652053656E736F727320696E737461C8
:109180006C6C65643A0925730A0043617061636918
:10919000746976652053656E736F72203120726535
:1091A0006164696E673A0925640A0043617061630E
:1091B00069746976652053656E736F722032207210
:1091C000656164696E673A0925640A000A436F6D38
:1091D0006D756E69636174696F6E20537461746933
:1091E00073746963733A0A0055415254312028451B
:1091F00078742E436F6D6D29204275666665722006
:109200004F76657272756E733A2025640A00554177
:109210005254322028496E742E436F6D6D292042BE
:109220007566666572204F76657272756E733A2048
:1092300025640A005541525433205B42542E436F3B
:109240006D6D5D20427566666572204F766572723F
:10925000756E733A2025640A000A536572766F2092
:1092600049447320696E2074686520496E74657284
:109270006E616C204275733A0A000A506F72742056
:109280007374617475733A0A00506F7274202564A8
:109290002043757272656E742052656164696E67F1
:1092A0003A204F5645524C4F4144204552524F525E
:1092B000202825646D41290A00506F7274202564AE
:1092C0002043757272656E742052656164696E67C1
:1092D0003A2025646D410A000A4120426C7565748C
:1092E0006F6F746820636F6D6D756E69636174690B
:1092F0006F6E206D6F64756C652069732070726588
:1093000073656E742E0A00426C7565746F6F7468B5
:1093100020706F776572207374617475733A2025BD
:10932000730A005365656420526F626F74696373DA
:109330002045524F53204669726D776172652C202B
:1093400076657273696F6E2025640A0A004C697332
:1093500074206F6620616476616E63656420636F5C
:109360006D6D616E64732E0A5741524E494E473AF5
:1093700020546865736520636F6D6D616E64732042
:1093800061726520726573657276656420666F72BE
:109390002074686520757365206F66205365656469
:1093A00020526F626F7469637320746563686E69BD
:1093B00063616C206167656E74732E0A496E636F1A
:1093C0007272656374207573616765206D617920C1
:1093D000636175736520696E6F7065726174696F22
:1093E0006E2C2064616D61676520616E64206D6123
:1093F0007920766F696420796F7572207761727257
:10940000616E74792E0A55736520617420796F75C9
:1094100072206F776E207269736B2E0A0A00616882
:10942000700954686973206D6573736167652E0AEE
:1094300000696E697420656570726F6D0A00696EEF
:10944000697420626F6172646D6F64656C205B6D1E
:109450006F64656C5D0A00696E697420626F617289
:10946000646877636F6E666967205B636F6E6669B9
:1094700067206D61736B5D0A00696E6974206375A6
:109480007272656E747265736973746F72205B7249
:1094900065736973746F722076616C7565204F68AF
:1094A0006D735D0A00696E697420736E205B595993
:1094B0005D205B4D4D5D205B434845434B53554D0F
:1094C0005D0A00696E69742073657269616C636F0F
:1094D0006D6D205B6C6566747C72696768745D0A8B
:1094E0000A005573652027636F6E666967272066DB
:1094F0006F72207468652072656D61696E696E6750
:1095000020636F6E66696775726174696F6E732E22
:109510002054797065202768656C702720666F720B
:1095200020696E666F726D6174696F6E2E0A0A0033
:109530004C697374206F6620617661696C61626C3E
:109540006520636F6D6D616E64732E20416C6C20BD
:10955000636F6D6D616E647320617265206361730A
:10956000652073656E7369746976652E0A0A0068F2
:10957000656C700954686973206D65737361676504
:109580002E0A0073746174757309446973706C6199
:10959000792063757272656E742073797374656D6A
:1095A000207374617475732E0A0061626F7574099B
:1095B000446973706C617920696E7465726E616C58
:1095C00020696E666F726D6174696F6E2E0A00732A
:1095D00063616E6275730952657363616E732074A3
:1095E000686520696E7465726E616C2062757320A7
:1095F000666F722044796E616D6978656C20646570
:1096000076696365732E0A006F70656E094F706529
:109610006E2068616E642E0A00636C6F7365094387
:109620006C6F73652068616E642E0A0070617274DD
:109630006F70656E205B76616C75653A20302D2504
:10964000645D095061727469616C6C79206F70653A
:109650006E2068616E642E0A00736574706F7320EB
:109660005B6465766963652069645D205B706F7318
:109670006974696F6E3A20302D25645D09536574F5
:1096800020706F736974696F6E20666F72207370DB
:1096900065636966696564206465766963652E0A39
:1096A0000072657374617274205B7073757C616C99
:1096B0006C5D095265737461727473206F6E6C799E
:1096C0002074686520736572766F20505355206F43
:1096D00072207468652066756C6C2073797374658C
:1096E0006D2E0A00636F6E666967205B6578746231
:1096F0006175647C65787469647C65787474786578
:109700006E61626C657C3132626974616463657834
:10971000706F7365647C696E74626175647C627479
:10972000626175647C62746E616D657C6274636F86
:1097300064657C6274636F6D6D616E645D205B76E1
:10974000616C75655D0A0953797374656D2077697D
:10975000646520636F6E66696775726174696F6EA8
:10976000206F7074696F6E732E0A00777262205BCF
:109770006465766963652069645D205B6164647219
:109780006573735D205B627974652076616C7565C5
:109790005D095772697465206279746520746F2061
:1097A0006465766963652E0A00777277205B64656D
:1097B000766963652069645D205B616464726573CA
:1097C000735D205B696E742076616C75655D095709
:1097D0007269746520776F726420746F2064657697
:1097E0006963652E0A00726562205B646576696351
:1097F000652069645D205B616464726573735D09F3
:109800005265616420627974652066726F6D2064B0
:1098100065766963652E0A00726577205B646576FC
:109820006963652069645D205B616464726573735C
:109830005D095265616420776F72642066726F6D96
:10984000206465766963652E0A0A00496E76616C4C
:10985000696420636F6D6D616E642E20436F6D6D62
:10986000616E647320617265206361736520736546
:109870006E7369746976652E0A547970652027685D
:10988000656C702720666F72206D6F726520696E3F
:10989000666F726D6174696F6E2E0A004944206EA6
:1098A0006F742070726573656E7420696E207468C1
:1098B0006520696E7465726E616C206275732E200E
:1098C0005479706520277374617475732720666FEF
:1098D000722061206C697374206F662076616C69F8
:1098E00064204944732E0A00496E76616C696420D5
:1098F000706F736974696F6E2E204D6178696D7534
:109900006D20616363657074656420706F73697442
:10991000696F6E20697320343039352E0A416374C3
:1099200075616C206D6178696D756D206465706519
:109930006E6473206F6E206163747561746F722042
:10994000636F6E66696775726174696F6E2E0A0067
:1099500070737500446F6E6500616C6C006578749F
:109960007478656E61626C6500796573006E6F0076
:1099700031326269746164636578706F7365640025
:10998000696E746261756400627462617564004935
:109990006E76616C69642073657474696E672E20DD
:1099A00053657474696E672073686F756C642062A8
:1099B000652061204261756420706172616D65741B
:1099C000657220286578616D706C653A2031363D8E
:1099D00031313532303062707329005375636573ED
:1099E0007320636F6E6669677572696E6720425493
:1099F000206D6F64756C652E0A004661696C656444
:109A000020636F6E6669677572696E6720425420C5
:109A10006D6F64756C652E0A005361766564207302
:109A2000657474696E6720696E204D61696E20628D
:109A30006F61726420656570726F6D2E0062746E66
:109A4000616D65005375636573730A004661696CE7
:109A50000A006274636F646500496E76616C6964C4
:109A600020636F64652E20436F6465206D75737489
:109A700020626520612034206469676974206E75F6
:109A80006D6572696320636F64652072616E6769DA
:109A90006E672066726F6D203030303020746F201A
:109AA000393939392E0A00537563636573732E2073
:109AB000425420636F64652073657420746F20279F
:109AC0002573272028616C77617973206120342009
:109AD000646967697420636F6465292E0A00627483
:109AE000636F6D6D616E64005265706C793A0A2522
:109AF000730A00656570726F6D00626F6172646DEC
:109B00006F64656C00626F6172646877636F6E6624
:109B100069670063757272656E74726573697374D8
:109B20006F720073657269616C636F6D6D006C6557
:109B3000667400726967687400736E0068656C70A3
:109B400000616870007374617475730061626F7591
:109B500074007363616E62757300636C6F7365008C
:109B6000706172746F70656E00736574706F7300EE
:109B70007265737461727400696E697400777262E1
:109B8000007772770072656200726577006D616CB4
:109B90006C6F63206661696C00636C734649464F65
:109BA0004C6973743A20617474656D7074656420D7
:109BB000746F2072656D6F7665206D6F72652069B8
:109BC00074656D73207468616E20776861742065B8
:109BD000786973747320696E20746865206C69738A
:109BE00074210043616C6C6F63206661696C006D69
:109BF000616C6C6F63206661696C203400FFFFFF4D
:109C00000000000000000000ED3C0000BD35000039
:109C1000F13500000000000000000000000000001E
:109C2000093F0000793D0000DD3D0000000000001C
:109C3000000000000100000002000000030000001E
:109C400004000000060000000700000008000000FB
:109C5000090000000A0000000B0000000C000000DA
:109C60000D0000000E0000000F00000010000000BA
:109C7000110000001200000013000000140000009A
:109C80001500000016000000180000001900000078
:109C90001A0000001B0000001C0000001D00000056
:109CA0001E0000001F000000200000002100000036
:109CB0002200000023000000240000002500000016
:109CC00026000000270000002800000029000000F6
:109CD0002A0000002B0000002C0000002D000000D6
:109CE0002E0000002F0000003000000031000000B6
:109CF0003200000033000000340000003500000096
:109D00003600000037000000380000003900000075
:109D10003A0000003B0000003C0000003D00000055
:109D20003E0000003F000000400000004100000035
:109D30004200000043000000440000004400000016
:109D400045000000460000004700000048000000F9
:109D5000490000004A0000004B0000004C000000D9
:109D60004D0000004E0000004F00000050000000B9
:109D70005100000052000000530000005400000099
:109D80005500000056000000570000005800000079
:109D900058000000590000005A0000005B0000005D
:109DA0005C0000005D0000005E0000005F0000003D
:109DB000600000006100000062000000630000001D
:109DC00064000000650000006600000066000000FE
:109DD0006700000068000000690000006A000000E1
:109DE0006B0000006C0000006D0000006E000000C1
:109DF0006F000000700000007100000072000000A1
:109E00007200000073000000740000007500000084
:109E10007600000077000000780000007900000064
:109E20007A0000007B0000007C0000007C00000045
:109E30007D0000007E0000007F0000008000000028
:109E40008100000082000000830000008400000008
:109E500085000000860000008600000087000000EA
:109E600088000000890000008A0000008B000000CC
:109E70008C0000008D0000008E0000008F000000AC
:109E80008F00000090000000910000009200000090
:109E90009300000094000000950000009600000070
:109EA0009700000097000000980000009900000053
:109EB0009A0000009B0000009C0000009D00000034
:109EC0009E0000009F0000009F000000A000000016
:109ED000A1000000A2000000A3000000A4000000F8
:109EE000A5000000A6000000A7000000A7000000D9
:109EF000A8000000A9000000AA000000AB000000BC
:109F0000AC000000AD000000AE000000AF0000009B
:109F1000AF000000B0000000B1000000B20000007F
:109F2000B3000000B4000000B5000000B60000005F
:109F3000B6000000B7000000B8000000B900000043
:109F4000BA000000BB000000BC000000BD00000023
:109F5000BE000000BE000000BF000000C000000006
:109F6000C1000000C2000000C3000000C4000000E7
:109F7000C5000000C5000000C6000000C7000000CA
:109F8000C8000000C9000000CA000000CB000000AB
:109F9000CC000000CD000000CD000000CE0000008D
:109FA000CF000000D0000000D1000000D20000006F
:109FB000D3000000D4000000D4000000D500000051
:109FC000D6000000D7000000D8000000D900000033
:109FD000DA000000DB000000DC000000DC00000014
:109FE000DD000000DE000000DF000000E0000000F7
:109FF000E1000000E2000000E3000000E4000000D7
:10A00000E4000000E5000000E6000000E7000000BA
:10A01000E8000000E9000000EA000000EB0000009A
:10A02000EB000000EC000000ED000000EE0000007E
:10A03000EF000000F0000000F1000000F20000005E
:10A04000F3000000F3000000F4000000F500000041
:10A05000F6000000F7000000F8000000F900000022
:10A06000FA000000FB000000FC000000FC00000003
:10A07000FD000000FE000000FF00000000010000E5
:10A0800001010000020100000301000004010000C2
:10A0900004010000050100000601000007010000A6
:10A0A00008010000090100000A0100000B01000086
:10A0B0000C0100000D0100000D0100000E01000068
:10A0C0000F0100001001000011010000120100004A
:10A0D000130100001401000015010000160100002A
:10A0E000170100001701000018010000190100000D
:10A0F0001A0100001B0100001C0100001D010000EE
:10A100001E0100001F0100002001000021010000CD
:10A1100021010000220100002301000024010000B1
:10A120002501000026010000270100002801000091
:10A13000290100002A0100002B0100002C01000071
:10A140002D0100002D0100002E0100002F01000054
:10A150003001000031010000320100003301000035
:10A160003401000035010000360100003701000015
:10A1700038010000390100003A0100003B010000F5
:10A180003B0100003C0100003D0100003E010000D9
:10A190003F010000400100004101000042010000B9
:10A1A0004301000044010000450100004601000099
:10A1B0004701000048010000490100004A01000079
:10A1C0004B0100004C0100004D0100004E01000059
:10A1D0004F0100004F01000050010000510100003C
:10A1E000520100005301000054010000550100001D
:10A1F00056010000570100005801000059010000FD
:10A200005A0100005B0100005C0100005D010000DC
:10A210005E0100005F0100006001000061010000BC
:10A22000620100006301000064010000650100009C
:10A23000660100006701000068010000690100007C
:10A240006A0100006B0100006C0100006D0100005C
:10A250006E0100006F01000070010000710100003C
:10A26000720100007301000074010000750100001C
:10A2700076010000770100007801000079010000FC
:10A280007A0100007B0100007C0100007D010000DC
:10A290007E0100007F0100008001000081010000BC
:10A2A000820100008301000084010000850100009C
:10A2B0008601000088010000890100008A01000079
:10A2C0008B0100008C0100008D0100008E01000058
:10A2D0008F01000090010000910100009201000038
:10A2E0009301000094010000950100009601000018
:10A2F00097010000980100009A0100009B010000F6
:10A300009C0100009D0100009E0100009F010000D3
:10A31000A0010000A1010000A2010000A3010000B3
:10A32000A4010000A6010000A7010000A801000090
:10A33000A9010000AA010000AB010000AC0100006F
:10A34000AD010000AE010000B0010000B10100004D
:10A35000B2010000B3010000B4010000B50100002B
:10A36000B6010000B7010000B9010000BA01000009
:10A37000BB010000BC010000BD010000BE010000E7
:10A38000C0010000C1010000C2010000C3010000C3
:10A39000C4010000C5010000C7010000C8010000A1
:10A3A000C9010000CA010000CB010000CC0100007F
:10A3B000CE010000CF010000D0010000D10100005B
:10A3C000D2010000D4010000D5010000D601000038
:10A3D000D7010000D8010000DA010000DB01000015
:10A3E000DC010000DD010000DF010000E0010000F1
:10A3F000E1010000E2010000E4010000E5010000CD
:10A40000E6010000E7010000E9010000EA010000A8
:10A41000EB010000EC010000EE010000EF01000084
:10A42000F0010000F2010000F3010000F40100005F
:10A43000F5010000F7010000F8010000F90100003B
:10A44000FB010000FC010000FD010000FF01000015
:10A4500000020000010200000302000004020000EC
:10A4600005020000070200000802000009020000C7
:10A470000B0200000C0200000D0200000F020000A1
:10A48000100200001202000013020000140200007B
:10A490001602000017020000190200001A02000054
:10A4A0001B0200001D0200001E020000200200002E
:10A4B0002102000023020000240200002602000006
:10A4C00027020000280200002A0200002B020000E0
:10A4D0002D0200002E0200003002000031020000B8
:10A4E0003302000034020000360200003702000090
:10A4F000390200003A0200003C0200003E02000067
:10A500003F0200004102000042020000440200003D
:10A510004502000047020000490200004A02000014
:10A520004C0200004D0200004F02000051020000EA
:10A5300052020000540200005602000057020000C0
:10A54000590200005B0200005C0200005E02000095
:10A55000600200006102000063020000650200006A
:10A5600066020000680200006A0200006C0200003F
:10A570006D0200006F020000710200007302000013
:10A580007402000076020000780200007A020000E7
:10A590007C0200007E0200007F02000081020000B9
:10A5A000830200008502000087020000890200008B
:10A5B0008B0200008D0200008E020000900200005D
:10A5C000920200009402000096020000980200002F
:10A5D0009A0200009C0200009E020000A0020000FF
:10A5E000A2020000A4020000A6020000A8020000CF
:10A5F000AB020000AD020000AF020000B10200009B
:10A60000B3020000B5020000B7020000B90200006A
:10A61000BC020000BE020000C0020000C202000036
:10A62000C4020000C7020000C9020000CB02000003
:10A63000CE020000D0020000D2020000D5020000CD
:10A64000D7020000D9020000DC020000DE02000098
:10A65000E1020000E3020000E5020000E802000061
:10A66000EA020000ED020000F0020000F202000029
:10A67000F5020000F7020000FA020000FC020000F0
:10A68000FF020000020300000503000007030000B2
:10A690000A0300000D030000100300001203000075
:10A6A00015030000180300001B0300001E03000038
:10A6B0002103000024030000270300002A030000F8
:10A6C0002D030000300300003303000036030000B8
:10A6D000390300003D030000400300004303000075
:10A6E000460300004A0300004D0300005003000031
:10A6F00054030000570300005B0300005E030000EA
:10A700006203000065030000690300006D030000A0
:10A710007103000074030000780300007C03000054
:10A720008003000084030000880300008C03000005
:10A730009003000094030000980300009D030000B4
:10A74000A1030000A5030000AA030000AE0300005F
:10A75000B3030000B8030000BC030000C103000005
:10A76000C6030000CB030000D0030000D5030000A7
:10A77000DA030000DF030000E5030000EA03000045
:10A78000EF030000F5030000FB03000000040000DD
:10A79000060400000C04000012040000190400006C
:10A7A0001F040000250400002C04000033040000F6
:10A7B0003A04000040040000480400004F04000078
:10A7C000560400005E040000660400006E040000F1
:10A7D000760400007E04000087040000900400005E
:10A7E00099040000A2040000AC040000B6040000BC
:10A7F000C0040000CA040000D5040000E00400000A
:10A80000EC040000F804000004050000110500003D
:10A810001E0500002C0500003A0500004905000057
:10A8200059050000690500007A0500008C0500004C
:10A830009F050000B3050000C8050000DE0500000C
:10A84000454550524F4D2077726974652064656E9E
:10A8500069656420627920696E7465726E616C202E
:10A8600070726F74656374696F6E2E204E72206F04
:10A87000662077726974657320617474656D707495
:10A88000656420696E2074686973207365737369E9
:10A890006F6E3A2000417474656D7074696E672044
:10A8A000746F207772697465206120424954206F6B
:10A8B0006E2061206269746D617020627574206918
:10A8C000742773206F7574206F662072616E6765E0
:10A8D0003B2074686520616C6C6F776564207261E1
:10A8E0006E676520697320307E372E00090AFFFFEE
:10A8F000FFFFFFFFFFFFFFFFFFFFFF0D0006080741
:10A90000FFFF0E0FFF0CFFFFFFFFFFFF0B05050E04
:10A9100008090D0C06070F04001303931A9217C5BC
:10A9200085848687C4FF6FF07F030370037813F07C
:10A93000800FFBD07047FFFF4008FE4340A004405B
:10A940004408FE4344A004400018FE4300C00440F5
:10A950003000FE43309004403400FE433490044005
:10A960001C18FE431CC004401018FE4310C00440D5
:10A970000818FE4308C004400C18FE430CC00440F5
:10A980000C10FE430CB004401010FE4310B0044005
:10A990001810FE4318B004401C10FE431CB00440C5
:10A9A0001410FE4314B004400418FE4304C00440D5
:10A9B0000010FE4300B004400008FE4300A0044025
:10A9C0000408FE4304A004400C08FE430CA004400D
:10A9D0000808FE4308A004401418FE4314C00440B5
:10A9E0001818FE4318C004400410FE4304B004408D
:10A9F0000810FE4308B004401400FE4314900440C5
:10AA00004C08FE434CA004400420FE4304D0044004
:10AA10002410FE4324B004402010FE4320B0044024
:10AA20002810FE4328B004402C10FE432CB00440F4
:10AA30000020FE4300D004404808FE4348A00440E4
:10AA40001000FE4310900440090AFFFFFFFFFFFFC4
:10AA5000FFFFFFFFFFFFFF0D00060807FFFF0E0FC0
:10AA6000FF0CFFFFFFFFFFFF0B05FFFFFFFFFFFFD7
:10AA70000000000000000000457100005D71000052
:10AA80002D71000035710000317100003971000036
:10AA9000D1700000E3700000037100000771000036
:10AAA0000D7100001D7100003D710000417100003A
:10AAB000A1700000AD700000B9700000C57000000A
:10AAC0006D710000517100000000000000000000E6
:10AAD000497200006172000031720000397200009A
:10AAE000357200003D720000D5710000E771000072
:10AAF000077200000B72000011720000217200004A
:10AB00004172000045720000A5710000B1710000A3
:10AB1000BD710000C9710000717200005572000023
:10AB200000000000000000004D730000657300008D
:10AB3000357300003D73000039730000417300005D
:10AB4000D9720000EB7200000B7300000F7300005D
:10AB50001573000025730000457300004973000061
:10AB6000A9720000B5720000C1720000CD72000031
:10AB700075730000597300000D0AFFFFFFFFFFFF10
:10AB80000000000000000000DB740000E174000021
:10AB9000CB740000CF740000D3740000D7740000A1
:10ABA00000151915000100007487FF1F1200000036
:10ABB000000200009E87FF1F43000000000300000A
:10ABC000F887FF1F00000000010309048687FF1FAC
:10ABD0000000000002030904E287FF1F00000000DC
:10ABE00003030904FC87FF1F0000000000000000B1
:10ABF00000000000000000004300FFFF1488FF1F5A
:10AC0000002020202020202020202828282828203C
:10AC10002020202020202020202020202020202034
:10AC2000208810101010101010101010101010109C
:10AC3000100404040404040404040410101010108C
:10AC40001010414141414141010101010101010156
:10AC500001010101010101010101010110101010A8
:10AC60001010424242424242020202020202020228
:10AC7000020202020202020202020202101010107C
:10AC800020000000000000000000000000000000A4
:10AC900000000000000000000000000000000000B4
:10ACA00000000000000000000000000000000000A4
:10ACB0000000000000000000000000000000000094
:10ACC0000000000000000000000000000000000084
:10ACD0000000000000000000000000000000000074
:10ACE0000000000000000000000000000000000064
:10ACF0000000000000000000000000000000000054
:10AD000000FFFFFF00000000000000000000000046
:10AD10000000000000000000000000000000000033
:10AD20000000000000000000000000000000000023
:10AD30000000000000000000000000000000000013
:10AD40000000000000000000000000000000000003
:10AD500000000000000000000000000000000000F3
:10AD600000000000232D302B2000686C4C0065662D
:10AD7000674546470030313233343536373839414C
:10AD80004243444546003031323334353637383962
:10AD900061626364656600FFF8B500BFF8BC08BC7B
:10ADA0009E46704735040000897100008D720000D6
:08ADB00091730000ED74000036
:10ADB800010000000A0400001091FF1F08000000B5
:10ADC800FFFFFFFF1201000202000040C0168304CB
:10ADD80000010102030118035400650065006E00BC
:10ADE800730079006400750069006E006F00090245
:10ADF8004300020100C03209040000010202010000
:10AE0800052400100105240101010424020605247B
:10AE18000600010705820310004009040100020A28
:10AE280000000007050302400000070584024000F7
:10AE3800000016035500530042002000530065002F
:10AE48007200690061006C00040309040C0300002F
:10AE580000000000000000000000000000000000EA
:10AE6800000000000000000004AD000024AD000058
:10AE780044AD0000000000000000000000000000D9
:10AE880000000000F8AB0000000000000000000017
:10AE980000000000000000000000000000000000AA
:10AEA800000000000000000000000000000000009A
:10AEB800000000000000000000000000000000008A
:0CAEC800000000001488FF1F00AC000018
:00000001FF
